Archive member included       because of file (symbol)

C:\agb\lib/libagbsyscall.a(AgbSysCpuSet.o)
                              m4aLib.o (CpuSet)
C:\agb\lib/libagbsyscall.a(AgbSysMidiKey2Freq.o)
                              E:\pm3sound20041208\pm3sound\SoundMon.o (MidiKey2Freq)
C:\agb\lib/libagbsyscall.a(AgbSysVBlankIntrWait.o)
                              E:\pm3sound20041208\pm3sound\SoundMon.o (VBlankIntrWait)
C:\Program Files\Cygnus\thumbelf-000512\H-i686-cygwin32\bin/../lib/gcc-lib/thumb-elf/2.9-arm-000512/libgcc.a(_call_via_rX.o)
                              m4aLib.o (_call_via_r1)
C:\Program Files\Cygnus\thumbelf-000512\H-i686-cygwin32\bin/../lib/gcc-lib/thumb-elf/2.9-arm-000512/libgcc.a(_divsi3.o)
                              m4aLib.o (__divsi3)
C:\Program Files\Cygnus\thumbelf-000512\H-i686-cygwin32\bin/../lib/gcc-lib/thumb-elf/2.9-arm-000512/libgcc.a(_dvmd_tls.o)
                              C:\Program Files\Cygnus\thumbelf-000512\H-i686-cygwin32\bin/../lib/gcc-lib/thumb-elf/2.9-arm-000512/libgcc.a(_divsi3.o) (__div0)
C:\Program Files\Cygnus\thumbelf-000512\H-i686-cygwin32\bin/../lib/gcc-lib/thumb-elf/2.9-arm-000512/libgcc.a(_modsi3.o)
                              E:\pm3sound20041208\pm3sound\SoundMon.o (__modsi3)
C:\Program Files\Cygnus\thumbelf-000512\H-i686-cygwin32\bin/../lib/gcc-lib/thumb-elf/2.9-arm-000512/libgcc.a(_udivsi3.o)
                              E:\pm3sound20041208\pm3sound\SoundMon.o (__udivsi3)
C:\Program Files\Cygnus\thumbelf-000512\H-i686-cygwin32\bin/../lib/gcc-lib/thumb-elf/2.9-arm-000512/libgcc.a(_umodsi3.o)
                              E:\pm3sound20041208\pm3sound\SoundMon.o (__umodsi3)
C:\Program Files\Cygnus\thumbelf-000512\H-i686-cygwin32\bin/../lib/gcc-lib/thumb-elf/2.9-arm-000512/../../../../thumb-elf/lib/libg.a(memcpy.o)
                              m4aLib.o (memcpy)

Allocating common symbols
Common symbol       size              file

c_bit               0x4               E:\pm3sound20041208\pm3sound\SoundMon.o
m4a_sound           0xfb0             m4aLib.o
p_rev               0x4               E:\pm3sound20041208\pm3sound\SoundMon.o
ImmSng              0x68              m4aLib.o
p_bit               0x4               E:\pm3sound20041208\pm3sound\SoundMon.o
ImmSngMA            0x80              m4aLib.o
c_mvg               0x4               E:\pm3sound20041208\pm3sound\SoundMon.o
AvrLinC             0x4               E:\pm3sound20041208\pm3sound\SoundMon.o
c_mvo               0x4               E:\pm3sound20041208\pm3sound\SoundMon.o
w_midibuf           0x4               E:\pm3sound20041208\pm3sound\SoundMon.o
vcount              0x4               E:\pm3sound20041208\pm3sound\SoundMon.o
m4a_mplay000        0x40              SoundDat.o
ExtMPlyJmpTbl       0x90              m4aLib.o
Cont                0x4               E:\pm3sound20041208\pm3sound\SoundMon.o
xcmdn               0x4               E:\pm3sound20041208\pm3sound\SoundMon.o
MaxLin              0x4               E:\pm3sound20041208\pm3sound\SoundMon.o
c_mch               0x4               E:\pm3sound20041208\pm3sound\SoundMon.o
AvrLinT             0x4               E:\pm3sound20041208\pm3sound\SoundMon.o
r_midibuf           0x4               E:\pm3sound20041208\pm3sound\SoundMon.o
Trg                 0x4               E:\pm3sound20041208\pm3sound\SoundMon.o
c_rev               0x4               E:\pm3sound20041208\pm3sound\SoundMon.o
sysex               0x4               E:\pm3sound20041208\pm3sound\SoundMon.o
m4a_cgbchn          0x100             m4aLib.o
MaxChnC             0x4               E:\pm3sound20041208\pm3sound\SoundMon.o
c_song              0x10              E:\pm3sound20041208\pm3sound\SoundMon.o
c_fre               0x4               E:\pm3sound20041208\pm3sound\SoundMon.o
p_mch               0x4               E:\pm3sound20041208\pm3sound\SoundMon.o
m4a_mplay001        0x40              SoundDat.o
m4a_mplay002        0x40              SoundDat.o
midibuf             0x100             E:\pm3sound20041208\pm3sound\SoundMon.o
IntrMainBuf         0x800             E:\pm3sound20041208\pm3sound\SoundMon.o
ImmSngTA            0x140             m4aLib.o
MaxChn              0x4               E:\pm3sound20041208\pm3sound\SoundMon.o
c_mpr               0x4               E:\pm3sound20041208\pm3sound\SoundMon.o
midi_ma             0x40              E:\pm3sound20041208\pm3sound\SoundMon.o
midi_ta             0x500             E:\pm3sound20041208\pm3sound\SoundMon.o
runst               0x4               E:\pm3sound20041208\pm3sound\SoundMon.o
PrsImmSng           0x34              m4aLib.o
KeyRep              0x4               E:\pm3sound20041208\pm3sound\SoundMon.o
OamBak              0x400             E:\pm3sound20041208\pm3sound\SoundMon.o
m4a_memacc_area     0x10              SoundDat.o
p_song              0x10              E:\pm3sound20041208\pm3sound\SoundMon.o
m4a_mplay003        0x40              SoundDat.o
p_fre               0x4               E:\pm3sound20041208\pm3sound\SoundMon.o
BgBak               0x800             E:\pm3sound20041208\pm3sound\SoundMon.o
CurtCurs            0x4               E:\pm3sound20041208\pm3sound\SoundMon.o

Memory Configuration

Name             Origin             Length             Attributes
*default*        0x00000000         0xffffffff

Linker script and memory map

LOAD E:\pm3sound20041208\pm3sound\crt0.o
LOAD m4aLib.o
LOAD E:\pm3sound20041208\pm3sound\SoundMon.o
LOAD E:\pm3sound20041208\pm3sound\SndMonDat.o
LOAD SoundDat.o
LOAD glockens_c5.o
LOAD porgan_c4.o
LOAD acobs_c1.o
LOAD slapbs_c1.o
LOAD synbs_c2.o
LOAD timpani_c2.o
LOAD octcho_c3.o
LOAD oboe_c3.o
LOAD oboe_c4.o
LOAD p_gt_c3.o
LOAD slapb_c1.o
LOAD vosne.o
LOAD woodat1.o
LOAD woodat2.o
LOAD bdrum.o
LOAD snare_l.o
LOAD hand_clap.o
LOAD oce_snare.o
LOAD tom.o
LOAD closehh.o
LOAD openhh.o
LOAD ride.o
LOAD tambo.o
LOAD splash.o
LOAD cymbal.o
LOAD h_conga.o
LOAD l_conga.o
LOAD ti_bass.o
LOAD rimshot.o
LOAD tom1.o
LOAD ridecap.o
LOAD cowbell.o
LOAD indian.o
LOAD triyang.o
LOAD suzu.o
LOAD kane.o
LOAD taiko.o
LOAD tsutsumi.o
LOAD piano1_c2.o
LOAD piano1_c3.o
LOAD piano1_c4.o
LOAD piano1_c6.o
LOAD str_c3.o
LOAD str_c4.o
LOAD str_c5.o
LOAD tr_c3.o
LOAD tr_c4.o
LOAD tr_c5.o
LOAD tuba_c1.o
LOAD tuba_c2.o
LOAD horn_c3.o
LOAD horn_c4.o
LOAD flute_c5.o
LOAD ebase_c1.o
LOAD koto_c4.o
LOAD shakuhachi_c4.o
LOAD koto_c3.o
LOAD ovgt_c3.o
LOAD disgt_c3.o
LOAD disgt_c2.o
LOAD gamelam_c3.o
LOAD pipeorg1_c3.o
LOAD pipeorg2_c4.o
LOAD voice_huu1.o
LOAD voice_haa1.o
LOAD elep4_c3.o
LOAD elep4_c4.o
LOAD tim_sn_c2.o
LOAD ban.o
LOAD psg_plus_c4.o
LOAD bic_bell.o
LOAD door.o
LOAD pizz_c4.o
LOAD track.o
LOAD moter.o
LOAD kaminari.o
LOAD kaze.o
LOAD bubble.o
LOAD iwa.o
LOAD fire.o
LOAD megab_c4.o
LOAD nami.o
LOAD gigigi.o
LOAD tu_bells_c4.o
LOAD bomb.o
LOAD big_bone_c2.o
LOAD harp_c5.o
LOAD xylophone_c5.o
LOAD kansei.o
LOAD tamakoro.o
LOAD accord_c4.o
LOAD voice_a.o
LOAD voice_i.o
LOAD voice_u.o
LOAD voice_e.o
LOAD voice_o.o
LOAD voice_n.o
LOAD pv001.o
LOAD pv002.o
LOAD pv003.o
LOAD pv004.o
LOAD pv005.o
LOAD pv006.o
LOAD pv007.o
LOAD pv008.o
LOAD pv009.o
LOAD pv010.o
LOAD pv011.o
LOAD pv012.o
LOAD pv013.o
LOAD pv014.o
LOAD pv015.o
LOAD pv016.o
LOAD pv017.o
LOAD pv018.o
LOAD pv019.o
LOAD pv020.o
LOAD pv021.o
LOAD pv022.o
LOAD pv023.o
LOAD pv024.o
LOAD pv025.o
LOAD pv026.o
LOAD pv027.o
LOAD pv028.o
LOAD pv029.o
LOAD pv030.o
LOAD pv031.o
LOAD pv032.o
LOAD pv033.o
LOAD pv034.o
LOAD pv035.o
LOAD pv036.o
LOAD pv037.o
LOAD pv038.o
LOAD pv039.o
LOAD pv040.o
LOAD pv041.o
LOAD pv042.o
LOAD pv043.o
LOAD pv044.o
LOAD pv045.o
LOAD pv046.o
LOAD pv047.o
LOAD pv048.o
LOAD pv049.o
LOAD pv050.o
LOAD pv051.o
LOAD pv052.o
LOAD pv053.o
LOAD pv054.o
LOAD pv055.o
LOAD pv056.o
LOAD pv057.o
LOAD pv058.o
LOAD pv059.o
LOAD pv060.o
LOAD pv061.o
LOAD pv062.o
LOAD pv063.o
LOAD pv064.o
LOAD pv065.o
LOAD pv066.o
LOAD pv067.o
LOAD pv068.o
LOAD pv069.o
LOAD pv070.o
LOAD pv071.o
LOAD pv072.o
LOAD pv073.o
LOAD pv074.o
LOAD pv075.o
LOAD pv076.o
LOAD pv077.o
LOAD pv078.o
LOAD pv079.o
LOAD pv080.o
LOAD pv081.o
LOAD pv082.o
LOAD pv083.o
LOAD pv084.o
LOAD pv085.o
LOAD pv086.o
LOAD pv087.o
LOAD pv088.o
LOAD pv089.o
LOAD pv090.o
LOAD pv091.o
LOAD pv092.o
LOAD pv093.o
LOAD pv094.o
LOAD pv095.o
LOAD pv096.o
LOAD pv097.o
LOAD pv098.o
LOAD pv099.o
LOAD pv100.o
LOAD pv101.o
LOAD pv102.o
LOAD pv103.o
LOAD pv104.o
LOAD pv105.o
LOAD pv106.o
LOAD pv107.o
LOAD pv108.o
LOAD pv109.o
LOAD pv110.o
LOAD pv111.o
LOAD pv112.o
LOAD pv113.o
LOAD pv114.o
LOAD pv115.o
LOAD pv116.o
LOAD pv117.o
LOAD pv118.o
LOAD pv119.o
LOAD pv120.o
LOAD pv121.o
LOAD pv122.o
LOAD pv123.o
LOAD pv124.o
LOAD pv125.o
LOAD pv126.o
LOAD pv127.o
LOAD pv128.o
LOAD pv129.o
LOAD pv130.o
LOAD pv131.o
LOAD pv132.o
LOAD pv133.o
LOAD pv134.o
LOAD pv135.o
LOAD pv136.o
LOAD pv137.o
LOAD pv138.o
LOAD pv139.o
LOAD pv140.o
LOAD pv141.o
LOAD pv142.o
LOAD pv143.o
LOAD pv144.o
LOAD pv145.o
LOAD pv146.o
LOAD pv147.o
LOAD pv148.o
LOAD pv149.o
LOAD pv150.o
LOAD pv151.o
LOAD pv152.o
LOAD pv153.o
LOAD pv154.o
LOAD pv155.o
LOAD pv156.o
LOAD pv157.o
LOAD pv158.o
LOAD pv159.o
LOAD pv160.o
LOAD pv161.o
LOAD pv162.o
LOAD pv163.o
LOAD pv164.o
LOAD pv165.o
LOAD pv166.o
LOAD pv167.o
LOAD pv168.o
LOAD pv169.o
LOAD pv170.o
LOAD pv171.o
LOAD pv172.o
LOAD pv173.o
LOAD pv174.o
LOAD pv175.o
LOAD pv176.o
LOAD pv177.o
LOAD pv178.o
LOAD pv179.o
LOAD pv180.o
LOAD pv181.o
LOAD pv182.o
LOAD pv183.o
LOAD pv184.o
LOAD pv185.o
LOAD pv186.o
LOAD pv187.o
LOAD pv188.o
LOAD pv189.o
LOAD pv190.o
LOAD pv191.o
LOAD pv192.o
LOAD pv193.o
LOAD pv194.o
LOAD pv195.o
LOAD pv196.o
LOAD pv197.o
LOAD pv198.o
LOAD pv199.o
LOAD pv200.o
LOAD pv201.o
LOAD pv202.o
LOAD pv203.o
LOAD pv204.o
LOAD pv205.o
LOAD pv206.o
LOAD pv207.o
LOAD pv208.o
LOAD pv209.o
LOAD pv210.o
LOAD pv211.o
LOAD pv212.o
LOAD pv213.o
LOAD pv214.o
LOAD pv215.o
LOAD pv216.o
LOAD pv217.o
LOAD pv218.o
LOAD pv219.o
LOAD pv220.o
LOAD pv221.o
LOAD pv222.o
LOAD pv223.o
LOAD pv224.o
LOAD pv225.o
LOAD pv226.o
LOAD pv227.o
LOAD pv228.o
LOAD pv229.o
LOAD pv230.o
LOAD pv231.o
LOAD pv232.o
LOAD pv233.o
LOAD pv234.o
LOAD pv235.o
LOAD pv236.o
LOAD pv237.o
LOAD pv238.o
LOAD pv239.o
LOAD pv240.o
LOAD pv241.o
LOAD pv242.o
LOAD pv243.o
LOAD pv244.o
LOAD pv245.o
LOAD pv246.o
LOAD pv247.o
LOAD pv248.o
LOAD pv249.o
LOAD pv250.o
LOAD pv251.o
LOAD pv252.o
LOAD pv253.o
LOAD pv254.o
LOAD pv255.o
LOAD pv256.o
LOAD pv257.o
LOAD pv258.o
LOAD pv259.o
LOAD pv260.o
LOAD pv261.o
LOAD pv262.o
LOAD pv263.o
LOAD pv264.o
LOAD pv265.o
LOAD pv266.o
LOAD pv267.o
LOAD pv268.o
LOAD pv269.o
LOAD pv270.o
LOAD pv271.o
LOAD pv272.o
LOAD pv273.o
LOAD pv274.o
LOAD pv275.o
LOAD pv276.o
LOAD pv277.o
LOAD pv278.o
LOAD pv279.o
LOAD pv280.o
LOAD pv281.o
LOAD pv282.o
LOAD pv283.o
LOAD pv284.o
LOAD pv285.o
LOAD pv286.o
LOAD pv287.o
LOAD pv288.o
LOAD pv289.o
LOAD pv290.o
LOAD pv291.o
LOAD pv292.o
LOAD pv293.o
LOAD pv294.o
LOAD pv295.o
LOAD pv296.o
LOAD pv297.o
LOAD pv298.o
LOAD pv299.o
LOAD pv300.o
LOAD pv301.o
LOAD pv302.o
LOAD pv303.o
LOAD pv304.o
LOAD pv305.o
LOAD pv306.o
LOAD pv307.o
LOAD pv308.o
LOAD pv309.o
LOAD pv310.o
LOAD pv311.o
LOAD pv312.o
LOAD pv313.o
LOAD pv314.o
LOAD pv315.o
LOAD pv316.o
LOAD pv317.o
LOAD pv318.o
LOAD pv319.o
LOAD pv320.o
LOAD pv321.o
LOAD pv322.o
LOAD pv323.o
LOAD pv324.o
LOAD pv325.o
LOAD pv326.o
LOAD pv327.o
LOAD pv328.o
LOAD pv329.o
LOAD pv330.o
LOAD pv331.o
LOAD pv332.o
LOAD pv333.o
LOAD pv334.o
LOAD pv335.o
LOAD pv336.o
LOAD pv337.o
LOAD pv338.o
LOAD pv339.o
LOAD pv340.o
LOAD pv341.o
LOAD pv342.o
LOAD pv343.o
LOAD pv344.o
LOAD pv345.o
LOAD pv346.o
LOAD pv347.o
LOAD pv348.o
LOAD pv349.o
LOAD pv350.o
LOAD pv351.o
LOAD pv352.o
LOAD pv353.o
LOAD pv354.o
LOAD pv355.o
LOAD pv356.o
LOAD pv357.o
LOAD pv358.o
LOAD pv359.o
LOAD pv360.o
LOAD pv361.o
LOAD pv362.o
LOAD pv363.o
LOAD pv364.o
LOAD pv365.o
LOAD pv366.o
LOAD pv367.o
LOAD pv368.o
LOAD pv369.o
LOAD pv370.o
LOAD pv371.o
LOAD pv372.o
LOAD pv373.o
LOAD pv374.o
LOAD pv375.o
LOAD pv376.o
LOAD pv377.o
LOAD pv378.o
LOAD pv379.o
LOAD pv380.o
LOAD pv381.o
LOAD pv382.o
LOAD pv383.o
LOAD pv384.o
LOAD pv385.o
LOAD pv386.o
LOAD pv387.o
LOAD pv388.o
LOAD shop.o
LOAD kiteki.o
LOAD a_guitar_c4.o
LOAD hau_c4.o
LOAD voice01_1.o
LOAD voice01_2.o
LOAD voice01_3.o
LOAD voice02_1.o
LOAD voice02_2.o
LOAD voice02_3.o
LOAD voice03_1.o
LOAD voice03_2.o
LOAD voice03_3.o
LOAD voice04_1.o
LOAD voice04_2.o
LOAD voice04_3.o
LOAD voice05_1.o
LOAD voice05_2.o
LOAD voice05_3.o
LOAD voice06_1.o
LOAD voice06_2.o
LOAD voice06_3.o
LOAD voice07_1.o
LOAD voice07_2.o
LOAD voice07_3.o
LOAD voice08_1.o
LOAD voice08_2.o
LOAD voice08_3.o
LOAD voice09_1.o
LOAD voice09_2.o
LOAD voice09_3.o
LOAD voice10_1.o
LOAD voice10_2.o
LOAD voice10_3.o
LOAD voice11_1.o
LOAD voice11_2.o
LOAD voice11_3.o
LOAD voice12_1.o
LOAD voice12_2.o
LOAD voice12_3.o
LOAD voice13_1.o
LOAD voice13_2.o
LOAD voice13_3.o
LOAD voice14_1.o
LOAD voice14_2.o
LOAD voice14_3.o
LOAD voice15_1.o
LOAD voice15_2.o
LOAD voice15_3.o
LOAD voice16_1.o
LOAD voice16_2.o
LOAD voice16_3.o
LOAD voice17_1.o
LOAD voice17_2.o
LOAD voice17_3.o
LOAD test_c4.o
LOAD stpia_c3.o
LOAD whis_c5.o
LOAD fue1.o
LOAD dummy.o
LOAD se_kaifuku.o
LOAD se_pc_login.o
LOAD se_pc_off.o
LOAD se_pc_on.o
LOAD se_select.o
LOAD se_win_open.o
LOAD se_wall_hit.o
LOAD se_door.o
LOAD se_kaidan.o
LOAD se_dansa.o
LOAD se_jitensya.o
LOAD se_kouka_l.o
LOAD se_kouka_m.o
LOAD se_kouka_h.o
LOAD se_bowa2.o
LOAD se_poke_dead.o
LOAD se_nigeru.o
LOAD se_jido_doa.o
LOAD se_naminori.o
LOAD se_ban.o
LOAD se_pin.o
LOAD se_boo.o
LOAD se_bowa.o
LOAD se_jyuni.o
LOAD se_a.o
LOAD se_i.o
LOAD se_u.o
LOAD se_e.o
LOAD se_o.o
LOAD se_n.o
LOAD se_seikai.o
LOAD se_hazure.o
LOAD se_exp.o
LOAD se_jite_pyoko.o
LOAD se_mu_pachi.o
LOAD se_tk_kasya.o
LOAD se_fu_zaku.o
LOAD se_fu_zaku2.o
LOAD se_fu_zuzuzu.o
LOAD se_ru_gashin.o
LOAD se_ru_gasyan.o
LOAD se_ru_bari.o
LOAD se_ru_hyuu.o
LOAD se_ki_gasyan.o
LOAD se_tk_warpin.o
LOAD se_tk_warpout.o
LOAD se_tu_saa.o
LOAD se_hi_turun.o
LOAD se_track_move.o
LOAD se_track_stop.o
LOAD se_track_haiki.o
LOAD se_track_door.o
LOAD se_moter.o
LOAD se_card.o
LOAD se_save.o
LOAD se_kon.o
LOAD se_kon2.o
LOAD se_kon3.o
LOAD se_kon4.o
LOAD se_suikomu.o
LOAD se_nageru.o
LOAD se_toy_c.o
LOAD se_toy_d.o
LOAD se_toy_e.o
LOAD se_toy_f.o
LOAD se_toy_g.o
LOAD se_toy_a.o
LOAD se_toy_b.o
LOAD se_toy_c1.o
LOAD se_mizu.o
LOAD se_hashi.o
LOAD se_daugi.o
LOAD se_pinpon.o
LOAD se_fuusen1.o
LOAD se_fuusen2.o
LOAD se_fuusen3.o
LOAD se_toy_kabe.o
LOAD se_toy_dango.o
LOAD se_doku.o
LOAD se_esuka.o
LOAD se_t_ame.o
LOAD se_t_ame_e.o
LOAD se_t_ooame.o
LOAD se_t_ooame_e.o
LOAD se_t_koame.o
LOAD se_t_koame_e.o
LOAD se_t_kami.o
LOAD se_t_kami2.o
LOAD se_elebeta.o
LOAD se_hinsi.o
LOAD se_expmax.o
LOAD se_tamakoro.o
LOAD se_tamakoro_e.o
LOAD se_basabasa.o
LOAD se_regi.o
LOAD se_c_gaji.o
LOAD se_c_maku_u.o
LOAD se_c_maku_d.o
LOAD se_c_pasi.o
LOAD se_c_syu.o
LOAD se_c_pikon.o
LOAD se_reapoke.o
LOAD se_op_basyu.o
LOAD se_bt_start.o
LOAD se_dendou.o
LOAD se_jihanki.o
LOAD se_tama.o
LOAD se_z_scroll.o
LOAD se_z_page.o
LOAD se_pn_on.o
LOAD se_pn_off.o
LOAD se_z_search.o
LOAD se_tamago.o
LOAD se_tb_start.o
LOAD se_tb_kon.o
LOAD se_tb_kara.o
LOAD se_bidoro.o
LOAD se_w085.o
LOAD se_w085b.o
LOAD se_w231.o
LOAD se_w171.o
LOAD se_w233.o
LOAD se_w233b.o
LOAD se_w145.o
LOAD se_w145b.o
LOAD se_w145c.o
LOAD se_w240.o
LOAD se_w015.o
LOAD se_w081.o
LOAD se_w081b.o
LOAD se_w088.o
LOAD se_w016.o
LOAD se_w016b.o
LOAD se_w003.o
LOAD se_w104.o
LOAD se_w013.o
LOAD se_w196.o
LOAD se_w086.o
LOAD se_w004.o
LOAD se_w025.o
LOAD se_w025b.o
LOAD se_w152.o
LOAD se_w026.o
LOAD se_w172.o
LOAD se_w172b.o
LOAD se_w053.o
LOAD se_w007.o
LOAD se_w092.o
LOAD se_w221.o
LOAD se_w221b.o
LOAD se_w052.o
LOAD se_w036.o
LOAD se_w059.o
LOAD se_w059b.o
LOAD se_w010.o
LOAD se_w011.o
LOAD se_w017.o
LOAD se_w019.o
LOAD se_w028.o
LOAD se_w013b.o
LOAD se_w044.o
LOAD se_w029.o
LOAD se_w057.o
LOAD se_w056.o
LOAD se_w250.o
LOAD se_w030.o
LOAD se_w039.o
LOAD se_w054.o
LOAD se_w077.o
LOAD se_w020.o
LOAD se_w082.o
LOAD se_w047.o
LOAD se_w195.o
LOAD se_w006.o
LOAD se_w091.o
LOAD se_w146.o
LOAD se_w120.o
LOAD se_w153.o
LOAD se_w071b.o
LOAD se_w071.o
LOAD se_w103.o
LOAD se_w062.o
LOAD se_w062b.o
LOAD se_w048.o
LOAD se_w187.o
LOAD se_w118.o
LOAD se_w155.o
LOAD se_w122.o
LOAD se_w060.o
LOAD se_w185.o
LOAD se_w014.o
LOAD se_w043.o
LOAD se_w207.o
LOAD se_w207b.o
LOAD se_w215.o
LOAD se_w109.o
LOAD se_w173.o
LOAD se_w280.o
LOAD se_w202.o
LOAD se_w060b.o
LOAD se_w076.o
LOAD se_w080.o
LOAD se_w100.o
LOAD se_w107.o
LOAD se_w166.o
LOAD se_w129.o
LOAD se_w115.o
LOAD se_w112.o
LOAD se_w197.o
LOAD se_w199.o
LOAD se_w236.o
LOAD se_w204.o
LOAD se_w268.o
LOAD se_w070.o
LOAD se_w063.o
LOAD se_w127.o
LOAD se_w179.o
LOAD se_w151.o
LOAD se_w201.o
LOAD se_w161.o
LOAD se_w161b.o
LOAD se_w227.o
LOAD se_w227b.o
LOAD se_w226.o
LOAD se_w208.o
LOAD se_w213.o
LOAD se_w213b.o
LOAD se_w234.o
LOAD se_w260.o
LOAD se_w328.o
LOAD se_w320.o
LOAD se_w255.o
LOAD se_w291.o
LOAD se_w089.o
LOAD se_w239.o
LOAD se_w230.o
LOAD se_w281.o
LOAD se_w327.o
LOAD se_w287.o
LOAD se_w257.o
LOAD se_w253.o
LOAD se_w258.o
LOAD se_w322.o
LOAD se_w298.o
LOAD se_w287b.o
LOAD se_w114.o
LOAD se_w063b.o
LOAD se_rg_w_door.o
LOAD se_rg_card1.o
LOAD se_rg_card2.o
LOAD se_rg_card3.o
LOAD se_rg_bag1.o
LOAD se_rg_bag2.o
LOAD se_rg_getting.o
LOAD se_rg_shop.o
LOAD se_rg_kiteki.o
LOAD se_rg_help_op.o
LOAD se_rg_help_cl.o
LOAD se_rg_help_ng.o
LOAD se_rg_deomov.o
LOAD se_rg_excellent.o
LOAD se_rg_nawamiss.o
LOAD se_toreeye.o
LOAD se_toreoff.o
LOAD se_hantei1.o
LOAD se_hantei2.o
LOAD se_curtain.o
LOAD se_curtain1.o
LOAD se_ussoki.o
LOAD tetsuji.o
LOAD field13.o
LOAD kachi22.o
LOAD kachi2.o
LOAD kachi3.o
LOAD kachi5.o
LOAD pcc.o
LOAD nibi.o
LOAD suikun.o
LOAD dooro1.o
LOAD dooro_x1.o
LOAD dooro_x3.o
LOAD machi_s2.o
LOAD machi_s4.o
LOAD gim.o
LOAD naminori.o
LOAD dan01.o
LOAD fanfa1.o
LOAD me_asa.o
LOAD me_bachi.o
LOAD fanfa4.o
LOAD fanfa5.o
LOAD me_waza.o
LOAD bijyutu.o
LOAD dooro_x4.o
LOAD fune_kan.o
LOAD me_shinka.o
LOAD shinka.o
LOAD me_wasure.o
LOAD syoujoeye.o
LOAD boyeye.o
LOAD dan02.o
LOAD machi_s3.o
LOAD odamaki.o
LOAD b_tower.o
LOAD swimeye.o
LOAD dan03.o
LOAD me_kinomi.o
LOAD me_tama.o
LOAD me_b_big.o
LOAD me_b_small.o
LOAD me_zannen.o
LOAD bd_time.o
LOAD test1.o
LOAD test2.o
LOAD test3.o
LOAD test4.o
LOAD test.o
LOAD gomachi0.o
LOAD gotown.o
LOAD pokecen.o
LOAD nextroad.o
LOAD granroad.o
LOAD cycling.o
LOAD friendly.o
LOAD mishiro.o
LOAD tozan.o
LOAD girleye.o
LOAD minamo.o
LOAD ashroad.o
LOAD event0.o
LOAD deepdeep.o
LOAD kachi1.o
LOAD title3.o
LOAD demo1.o
LOAD girl_sup.o
LOAD hageshii.o
LOAD kakkoii.o
LOAD kazanbai.o
LOAD aqa_0.o
LOAD tsuretek.o
LOAD boy_sup.o
LOAD rainbow.o
LOAD ayasii.o
LOAD kachi4.o
LOAD ropeway.o
LOAD casino.o
LOAD hightown.o
LOAD safari.o
LOAD c_road.o
LOAD ajito.o
LOAD m_boat.o
LOAD m_dungon.o
LOAD finecity.o
LOAD machupi.o
LOAD p_school.o
LOAD dendou.o
LOAD tonekusa.o
LOAD maborosi.o
LOAD con_fan.o
LOAD contest0.o
LOAD mgm0.o
LOAD t_battle.o
LOAD ooame.o
LOAD hideri.o
LOAD runecity.o
LOAD con_k.o
LOAD eikou_r.o
LOAD karakuri.o
LOAD hutago.o
LOAD sitennou.o
LOAD yama_eye.o
LOAD conlobby.o
LOAD inter_v.o
LOAD daigo.o
LOAD thankfor.o
LOAD end.o
LOAD mus_b_frontier.o
LOAD mus_b_arena.o
LOAD me_pointget.o
LOAD me_tore_eye.o
LOAD mus_pyramid.o
LOAD mus_pyramid_top.o
LOAD mus_b_palace.o
LOAD mus_rekkuu_kourin.o
LOAD mus_sattower.o
LOAD me_symbolget.o
LOAD mus_b_dome.o
LOAD mus_b_tube.o
LOAD mus_b_factory.o
LOAD mus_vs_rekku.o
LOAD mus_vs_front.o
LOAD mus_vs_mew.o
LOAD mus_b_dome1.o
LOAD battle27.o
LOAD battle31.o
LOAD battle20.o
LOAD battle32.o
LOAD battle33.o
LOAD battle36.o
LOAD battle34.o
LOAD battle35.o
LOAD battle38.o
LOAD battle30.o
LOAD mus_rg_annai.o
LOAD mus_rg_slot.o
LOAD mus_rg_ajito.o
LOAD mus_rg_gym.o
LOAD mus_rg_purin.o
LOAD mus_rg_demo.o
LOAD mus_rg_title.o
LOAD mus_rg_guren.o
LOAD mus_rg_shion.o
LOAD mus_rg_kaihuku.o
LOAD mus_rg_cycling.o
LOAD mus_rg_rocket.o
LOAD mus_rg_shoujo.o
LOAD mus_rg_shounen.o
LOAD mus_rg_dendou.o
LOAD mus_rg_t_mori.o
LOAD mus_rg_otsukimi.o
LOAD mus_rg_pokeyashi.o
LOAD mus_rg_ending.o
LOAD mus_rg_load01.o
LOAD mus_rg_opening.o
LOAD mus_rg_load02.o
LOAD mus_rg_load03.o
LOAD mus_rg_champ_r.o
LOAD mus_rg_vs_gym.o
LOAD mus_rg_vs_tore.o
LOAD mus_rg_vs_yasei.o
LOAD mus_rg_vs_last.o
LOAD mus_rg_masara.o
LOAD mus_rg_kenkyu.o
LOAD mus_rg_ohkido.o
LOAD mus_rg_pokecen.o
LOAD mus_rg_santoan.o
LOAD mus_rg_naminori.o
LOAD mus_rg_p_tower.o
LOAD mus_rg_shiruhu.o
LOAD mus_rg_hanada.o
LOAD mus_rg_tamamusi.o
LOAD mus_rg_win_tre.o
LOAD mus_rg_win_yasei.o
LOAD mus_rg_win_gym.o
LOAD mus_rg_kuchiba.o
LOAD mus_rg_nibi.o
LOAD mus_rg_rival1.o
LOAD mus_rg_rival2.o
LOAD mus_rg_fan2.o
LOAD mus_rg_fan5.o
LOAD mus_rg_fan6.o
LOAD me_rg_photo.o
LOAD mus_rg_titlerog.o
LOAD mus_rg_get_yasei.o
LOAD mus_rg_sousa.o
LOAD mus_rg_sekaikan.o
LOAD mus_rg_seibetu.o
LOAD mus_rg_jump.o
LOAD mus_rg_union.o
LOAD mus_rg_network.o
LOAD mus_rg_okurimono.o
LOAD mus_rg_kinomikui.o
LOAD mus_rg_nanadungeon.o
LOAD mus_rg_oshie_tv.o
LOAD mus_rg_nanashima.o
LOAD mus_rg_nanaiseki.o
LOAD mus_rg_nana123.o
LOAD mus_rg_nana45.o
LOAD mus_rg_nana67.o
LOAD mus_rg_pokefue.o
LOAD mus_rg_vs_deo.o
LOAD mus_rg_vs_myu2.o
LOAD mus_rg_vs_den.o
LOAD mus_rg_exeye.o
LOAD mus_rg_deoeye.o
LOAD mus_rg_t_tower.o
LOAD mus_rg_slowmasara.o
LOAD mus_rg_tvnoize.o
LOAD seq_01_1.o
LOAD seq_01_2.o
LOAD seq_01_3.o
LOAD seq_02_1.o
LOAD seq_02_2.o
LOAD seq_02_3.o
LOAD seq_03_1.o
LOAD seq_03_2.o
LOAD seq_03_3.o
LOAD seq_04_1.o
LOAD seq_04_2.o
LOAD seq_04_3.o
LOAD seq_05_1.o
LOAD seq_05_2.o
LOAD seq_05_3.o
LOAD seq_06_1.o
LOAD seq_06_2.o
LOAD seq_06_3.o
LOAD seq_07_1.o
LOAD seq_07_2.o
LOAD seq_07_3.o
LOAD seq_08_1.o
LOAD seq_08_2.o
LOAD seq_08_3.o
LOAD seq_09_1.o
LOAD seq_09_2.o
LOAD seq_09_3.o
LOAD seq_10_1.o
LOAD seq_10_2.o
LOAD seq_10_3.o
LOAD seq_11_1.o
LOAD seq_11_2.o
LOAD seq_11_3.o
LOAD seq_12_1.o
LOAD seq_12_2.o
LOAD seq_12_3.o
LOAD seq_13_1.o
LOAD seq_13_2.o
LOAD seq_13_3.o
LOAD seq_14_1.o
LOAD seq_14_2.o
LOAD seq_14_3.o
LOAD seq_15_1.o
LOAD seq_15_2.o
LOAD seq_15_3.o
LOAD seq_16_1.o
LOAD seq_16_2.o
LOAD seq_16_3.o
LOAD seq_17_1.o
LOAD seq_17_2.o
LOAD seq_17_3.o
LOAD C:\agb\lib/libagbsyscall.a
LOAD C:\Program Files\Cygnus\thumbelf-000512\H-i686-cygwin32\bin/../lib/gcc-lib/thumb-elf/2.9-arm-000512/libgcc.a
LOAD C:\Program Files\Cygnus\thumbelf-000512\H-i686-cygwin32\bin/../lib/gcc-lib/thumb-elf/2.9-arm-000512/../../../../thumb-elf/lib/libg.a
LOAD C:\Program Files\Cygnus\thumbelf-000512\H-i686-cygwin32\bin/../lib/gcc-lib/thumb-elf/2.9-arm-000512/../../../../thumb-elf/lib/libc.a
LOAD C:\Program Files\Cygnus\thumbelf-000512\H-i686-cygwin32\bin/../lib/gcc-lib/thumb-elf/2.9-arm-000512/libgcc.a
Address of section .text set to 0x8000000
Address of section .bss set to 0x3000000
                0x00008000                .=0x8000

.interp
 *(.interp)

.hash
 *(.hash)

.dynsym
 *(.dynsym)

.dynstr
 *(.dynstr)

.gnu.version
 *(.gnu.version)

.gnu.version_d
 *(.gnu.version_d)

.gnu.version_r
 *(.gnu.version_r)

.rel.text
 *(.rel.text)
 *(.rel.text.*)
 *(.rel.gnu.linkonce.t*)

.rela.text
 *(.rela.text)
 *(.rela.text.*)
 *(.rela.gnu.linkonce.t*)

.rel.data
 *(.rel.data)
 *(.rel.data.*)
 *(.rel.gnu.linkonce.d*)

.rela.data
 *(.rela.data)
 *(.rela.data.*)
 *(.rela.gnu.linkonce.d*)

.rel.rodata
 *(.rel.rodata)
 *(.rel.rodata.*)
 *(.rel.gnu.linkonce.r*)

.rela.rodata
 *(.rela.rodata)
 *(.rela.rodata.*)
 *(.rela.gnu.linkonce.r*)

.rel.got
 *(.rel.got)

.rela.got
 *(.rela.got)

.rel.ctors
 *(.rel.ctors)

.rela.ctors
 *(.rela.ctors)

.rel.dtors
 *(.rel.dtors)

.rela.dtors
 *(.rela.dtors)

.rel.init
 *(.rel.init)

.rela.init
 *(.rela.init)

.rel.fini
 *(.rel.fini)

.rela.fini
 *(.rela.fini)

.rel.bss
 *(.rel.bss)

.rela.bss
 *(.rela.bss)

.rel.plt
 *(.rel.plt)

.rela.plt
 *(.rela.plt)

.init
 *(.init)

.plt
 *(.plt)

.text           0x08000000     0x4578
 *(.text)
 .text          0x08000000      0x1d0 E:\pm3sound20041208\pm3sound\crt0.o
                0x080001d0                seg_m4aLib_top
                0x08000000                _start
                0x080000c0                start_vector
                0x080000fc                intr_main
 .text          0x080001d0     0x2810 m4aLib.o
                0x080028f4                pokVoicePitch
                0x080018e8                SoundVSyncOff_rev01
                0x08001758                SampFreqSet_rev01
                0x080001d0                umul3232H32
                0x0800151c                MPlayExtender
                0x08001894                SoundClear_rev01
                0x08002950                pokVoiceCheck
                0x080026fc                ply_xsust
                0x0800164c                Clear64byte_rev
                0x080026e8                ply_xdeca
                0x08001634                MusicPlayerJumpTableCopy
                0x080026c0                ply_xtype
                0x080022a0                MPlayVolumeControl
                0x08001a18                MPlayStart_rev01
                0x08000968                SoundMainBTM
                0x080027f8                pokVoiceStart
                0x08002750                ply_xswee
                0x08001964                SoundVSyncOn_rev01
                0x0800147c                m4aMPlayFadeOut
                0x08002968                pokVoiceChorus
                0x080019a0                MPlayOpen_rev01
                0x08000e48                TrackStop_rev01
                0x08001438                m4aMPlayAllContinue
                0x080026d4                ply_xatta
                0x08001cb8                MidiKey2CgbFr
                0x08002724                ply_xiecv
                0x080013b4                m4aSongNumContinue
                0x08002478                MPlayLFOSpeedSet
                0x080011b4                DummyFunc
                0x08002944                pokVoiceProgress
                0x0800148c                m4aMPlayFadeOutPause
                0x080011d4                MPlayFadeOut
                0x080010c0                ply_endtie_rev01
                0x0800142c                m4aMPlayContinue
                0x08002278                MPlayTempoControl
                0x08001b3c                FadeOutBody_rev01
                0x08001d60                CgbOscOff
                0x08002664                ply_xxx
                0x08002994                pokStereoMono
                0x08001150                MidiKey2fr
                0x080012a8                m4aSoundMain
                0x08002678                ply_xwave
                0x08001c04                TrkVolPitSet_rev01
                0x080014ac                m4aMPlayFadeInContinue
                0x080012b4                m4aSongNumStart
                0x08001128                ply_lfos_rev01
                0x080011b8                MPlayContinue
                0x0800113c                ply_mod_rev01
                0x08002308                MPlayPitchControl
                0x080023e4                MP_clear_modM
                0x08000be0                MPlayMain_rev01
                0x08000ebc                ply_note_rev01
                0x08001660                SoundInit_rev01
                0x080012e0                m4aSongNumStartOrChange
                0x080028c8                pokVoiceVolume
                0x08002404                MPlayModDepthSet
                0x0800132c                m4aSongNumStartOrContinue
                0x08002764                ply_xwait
                0x08001e2c                CgbSound
                0x08001afc                MPlayStop_rev01
                0x080027f4                DummyFunc_rev
                0x08002644                ply_xcmd
                0x080017fc                SoundMode_rev01
                0x08002938                pokVoiceRelease
                0x080027ac                ply_xadct
                0x0800237c                MPlayPanpotControl
                0x08001638                ClearChain_rev
                0x08000b94                SoundVSync_rev01
                0x0800292c                pokVoiceLength
                0x080011f4                m4aSoundInit
                0x08002730                ply_xiecl
                0x0800273c                ply_xleng
                0x080014d4                m4aMPlayImmInit
                0x080024ec                ply_memacc
                0x080001e0                SoundMain
                0x080028dc                pokVoicePanpot
                0x08000264                SoundMainRAM
                0x080029d4                pokVoicePriority
                0x080013e8                m4aMPlayAllStop
                0x08001db0                CgbModVol
                0x08000968                Clear64byte
                0x08001380                m4aSongNumStop
                0x080009d0                MPlyJmpTblCopy
                0x08002710                ply_xrele
 .text          0x080029e0     0x184c E:\pm3sound20041208\pm3sound\SoundMon.o
                0x08003098                IntrDummy
                0x08003868                ModeWrite
                0x080032f0                ValueChangePlus
                0x08003084                VBlankIntr
                0x08003544                ValueWrite
                0x08003bc8                MidiInputMain
                0x080029e0                seg_m4aLib_end
                0x08003bb0                unReadMidi
                0x08003024                KeyRead
                0x08003920                MidiWrite
                0x08003b18                MidiInIntr
                0x08003668                SongWrite
                0x080041f0                MidiAllStop
                0x0800309c                ValueChange
                0x080029e4                _MPlayFadeOut
                0x0800351c                StrWrite
                0x08003ae4                MidiPortInit
                0x080039c4                MidiInputInit
                0x080035d8                ValueWriteHex
                0x08003b78                ReadMidi
                0x080029e8                AgbMain
 .text          0x0800422c        0x4 C:\agb\lib/libagbsyscall.a(AgbSysCpuSet.o)
                0x0800422c                CpuSet
 .text          0x08004230        0x4 C:\agb\lib/libagbsyscall.a(AgbSysMidiKey2Freq.o)
                0x08004230                MidiKey2Freq
 .text          0x08004234        0x8 C:\agb\lib/libagbsyscall.a(AgbSysVBlankIntrWait.o)
                0x08004234                VBlankIntrWait
 .text          0x0800423c       0x3c C:\Program Files\Cygnus\thumbelf-000512\H-i686-cygwin32\bin/../lib/gcc-lib/thumb-elf/2.9-arm-000512/libgcc.a(_call_via_rX.o)
                0x08004244                _call_via_r2
                0x08004254                _call_via_r6
                0x08004250                _call_via_r5
                0x08004248                _call_via_r3
                0x08004268                _call_via_fp
                0x0800425c                _call_via_r8
                0x08004258                _call_via_r7
                0x0800423c                _call_via_r0
                0x08004264                _call_via_sl
                0x08004270                _call_via_sp
                0x08004260                _call_via_r9
                0x0800424c                _call_via_r4
                0x08004240                _call_via_r1
                0x0800426c                _call_via_ip
                0x08004274                _call_via_lr
 .text          0x08004278       0x94 C:\Program Files\Cygnus\thumbelf-000512\H-i686-cygwin32\bin/../lib/gcc-lib/thumb-elf/2.9-arm-000512/libgcc.a(_divsi3.o)
                0x08004278                __divsi3
 .text          0x0800430c        0x4 C:\Program Files\Cygnus\thumbelf-000512\H-i686-cygwin32\bin/../lib/gcc-lib/thumb-elf/2.9-arm-000512/libgcc.a(_dvmd_tls.o)
                0x0800430c                __div0
 .text          0x08004310       0xd0 C:\Program Files\Cygnus\thumbelf-000512\H-i686-cygwin32\bin/../lib/gcc-lib/thumb-elf/2.9-arm-000512/libgcc.a(_modsi3.o)
                0x08004310                __modsi3
 .text          0x080043e0       0x78 C:\Program Files\Cygnus\thumbelf-000512\H-i686-cygwin32\bin/../lib/gcc-lib/thumb-elf/2.9-arm-000512/libgcc.a(_udivsi3.o)
                0x080043e0                __udivsi3
 .text          0x08004458       0xc0 C:\Program Files\Cygnus\thumbelf-000512\H-i686-cygwin32\bin/../lib/gcc-lib/thumb-elf/2.9-arm-000512/libgcc.a(_umodsi3.o)
                0x08004458                __umodsi3
 .text          0x08004518       0x60 C:\Program Files\Cygnus\thumbelf-000512\H-i686-cygwin32\bin/../lib/gcc-lib/thumb-elf/2.9-arm-000512/../../../../thumb-elf/lib/libg.a(memcpy.o)
                0x08004518                memcpy
 *(.text.*)
 *(.stub)
 *(.gnu.warning)
 *(.gnu.linkonce.t*)
 *(.glue_7t)
 *(.glue_7)
                0x08004578                _etext=.
                0x08004578                PROVIDE (etext, .)

.fini
 *(.fini)

.rodata         0x08004578   0x32fa94
 *(.rodata)
 .rodata        0x08004578        0x4 E:\pm3sound20041208\pm3sound\crt0.o
                0x0800457c                seg_m4aLib_rodata_top
 .rodata        0x0800457c      0x324 m4aLib.o
                0x080046d0                FreqTable
                0x08004834                IniImmSng
                0x0800479c                CgbFrTable
                0x0800457c                MPlyJmpTbl
                0x080047f0                Cgb3vol
                0x0800461c                ScaleTable
                0x08004868                xcmd_tbl
                0x08004800                clock_tbl_rev01
                0x08004718                CgbScTable
                0x080047b4                NoiseTable
                0x08004700                pcmVBtbl_rev
 .rodata        0x080048a0     0x13c0 E:\pm3sound20041208\pm3sound\SoundMon.o
                0x08005bf4                IntrTable
                0x08004dec                OamData_Sample
                0x080048a0                seg_m4aLib_rodata_end
                0x080048bc                CurP
                0x08004df4                PlttData_Sample
                0x080048a2                FreTbl
                0x08004ff4                CharData_Sample
                0x080048ec                BgScData_Sample
 .rodata        0x08005c60     0x105c E:\pm3sound20041208\pm3sound\SndMonDat.o
                0x080065e8                app_vgrp_table
                0x08006cbc                seg_rodata_top
                0x08005c60                app_song_table
 .rodata        0x08006cbc    0x40000 SoundDat.o
                0x08013688                voicegroup061
                0x08044804                voicegroup434
                0x0803daf0                voicegroup386
                0x08009ddc                voicegroup026
                0x08018c2c                voicegroup077
                0x0800ad78                voicegroup030
                0x0802e0ac                voicegroup190
                0x0800d9a0                voicegroup041
                0x0801da2c                voicegroup090
                0x08007a78                voicegroup006
                0x0801802c                voicegroup075
                0x0800cd58                voicegroup038
                0x08039818                voicegroup374
                0x080381f8                voicegroup370
                0x08035bac                voicegroup363
                0x08027a28                voicegroup119
                0x0800f2cc                voicegroup047
                0x08013c88                voicegroup062
                0x0802960c                voicegroup124
                0x08009f38                voicegroup027
                0x08008fa8                voicegroup023
                0x0801fc34                voicegroup097
                0x0801c22c                voicegroup086
                0x08006cbc                voicegroup000
                0x08027044                voicegroup117
                0x08023834                voicegroup107
                0x080335a8                voicegroup355
                0x0803458c                voicegroup358
                0x0801862c                voicegroup076
                0x0800d13c                voicegroup039
                0x08043604                voicegroup431
                0x0803e0f0                voicegroup387
                0x08040e80                voicegroup397
                0x0800eccc                voicegroup046
                0x08041fa8                voicegroup402
                0x0801169c                voicegroup055
                0x080361ac                voicegroup364
                0x0802bc28                voicegroup152
                0x08010cd0                voicegroup053
                0x08040724                voicegroup394
                0x0801aa2c                voicegroup082
                0x0803a874                voicegroup377
                0x08014000                voicegroup063
                0x08023234                voicegroup106
                0x08020834                voicegroup099
                0x0800a37c                voicegroup028
                0x0800fad0                voicegroup050
                0x0801bc2c                voicegroup085
                0x08030adc                voicegroup206
                0x0803ecf0                voicegroup389
                0x08041b88                voicegroup401
                0x0803be94                voicegroup381
                0x0800d55c                voicegroup040
                0x08032570                voicegroup352
                0x08034b8c                voicegroup359
                0x08007a48                voicegroup005
                0x08028628                voicegroup121
                0x08021a34                voicegroup102
                0x0803c8f0                voicegroup383
                0x08016a00                voicegroup070
                0x08039c74                voicegroup375
                0x0803ba74                voicegroup380
                0x0800b6fc                voicegroup033
                0x0803170c                voicegroup301
                0x08037d9c                voicegroup369
                0x080097dc                voicegroup025
                0x08013088                voicegroup060
                0x08015800                voicegroup067
                0x08012c68                voicegroup059
                0x08015e00                voicegroup068
                0x0802a20c                voicegroup126
                0x08024a34                voicegroup110
                0x0802c8b8                voicegroup155
                0x0800e0fc                voicegroup043
                0x08007ac0                voicegroup008
                0x080304dc                voicegroup205
                0x0801b02c                voicegroup083
                0x0803a274                voicegroup376
                0x0801ec2c                voicegroup093
                0x0802c4b0                voicegroup154
                0x08027428                voicegroup118
                0x0802b7e4                voicegroup151
                0x0803c494                voicegroup382
                0x0802ae0c                voicegroup128
                0x08040d24                voicegroup395
                0x08022034                voicegroup103
                0x080414e0                voicegroup399
                0x08016e2c                voicegroup072
                0x08015200                voicegroup066
                0x080084e0                voicegroup021
                0x0802e6ac                voicegroup191
                0x08041768                voicegroup400
                0x0800bf6c                voicegroup035
                0x08028028                voicegroup120
                0x0802f2ac                voicegroup201
                0x08014600                voicegroup064
                0x0800a97c                voicegroup029
                0x08022c34                voicegroup105
                0x080367ac                voicegroup365
                0x08038c18                voicegroup372
                0x080357bc                voicegroup362
                0x08012668                voicegroup058
                0x0801d42c                voicegroup089
                0x08007538                voicegroup003
                0x08040124                voicegroup393
                0x0802f8ac                voicegroup202
                0x0801742c                voicegroup073
                0x0800e8d0                voicegroup045
                0x0801f634                voicegroup096
                0x080080d8                voicegroup010
                0x0800c35c                voicegroup036
                0x08023e34                voicegroup108
                0x08022634                voicegroup104
                0x0802fedc                voicegroup204
                0x0800b18c                voicegroup031
                0x08014c00                voicegroup065
                0x08044204                voicegroup433
                0x08040e50                voicegroup396
                0x08029c0c                voicegroup125
                0x08012068                voicegroup057
                0x0800e4e0                voicegroup044
                0x080080c0                voicegroup009
                0x08028a0c                voicegroup122
                0x0800dafc                voicegroup042
                0x08007a9c                voicegroup007
                0x0802a80c                voicegroup127
                0x0801a42c                voicegroup081
                0x080431fc                voicegroup430
                0x080080f0                voicegroup020
                0x080106d0                voicegroup052
                0x0803d4f0                voicegroup385
                0x0801e02c                voicegroup091
                0x080351bc                voicegroup361
                0x080425a8                voicegroup403
                0x0803f2f0                voicegroup390
                0x080412a0                voicegroup398
                0x08033170                voicegroup354
                0x080100d0                voicegroup051
                0x080310dc                voicegroup207
                0x0802feac                voicegroup203
                0x0802c06c                voicegroup153
                0x0802cca8                voicegroup156
                0x08025034                voicegroup111
                0x0801ce2c                voicegroup088
                0x0800b5a0                voicegroup032
                0x080427dc                voicegroup404
                0x0801f244                voicegroup095
                0x080072b0                voicegroup002
                0x0802b40c                voicegroup150
                0x08036dac                voicegroup366
                0x0803518c                voicegroup360
                0x08026b34                voicegroup116
                0x0803ae74                voicegroup378
                0x0800bb28                voicegroup034
                0x08019e2c                voicegroup080
                0x08045404                voicegroup436
                0x0803e6f0                voicegroup388
                0x0801922c                voicegroup078
                0x08031f70                voicegroup351
                0x0801982c                voicegroup079
                0x08043c04                voicegroup432
                0x08039218                voicegroup373
                0x0801b62c                voicegroup084
                0x08021434                voicegroup101
                0x0801e62c                voicegroup092
                0x080373ac                voicegroup367
                0x08020e34                voicegroup100
                0x08025634                voicegroup112
                0x08026534                voicegroup115
                0x08024434                voicegroup109
                0x08017a2c                voicegroup074
                0x0803779c                voicegroup368
                0x0802d2a8                voicegroup157
                0x0800c758                voicegroup037
                0x080077c0                voicegroup004
                0x08044e04                voicegroup435
                0x0801ec44                voicegroup094
                0x0803110c                voicegroup300
                0x0802615c                voicegroup114
                0x0802daac                voicegroup159
                0x0803fb24                voicegroup392
                0x0802ecac                voicegroup200
                0x080387f8                voicegroup371
                0x08016400                voicegroup069
                0x080093e0                voicegroup024
                0x08033f8c                voicegroup357
                0x08020234                voicegroup098
                0x0803cef0                voicegroup384
                0x0801c82c                voicegroup087
                0x08007154                voicegroup001
                0x08031970                voicegroup350
                0x08032b70                voicegroup353
                0x08011a68                voicegroup056
                0x0803398c                voicegroup356
                0x0800f6f8                voicegroup048
                0x08025c34                voicegroup113
                0x08045978                mplay_table
                0x0802d6bc                voicegroup158
                0x0802900c                voicegroup123
                0x08008ae0                voicegroup022
                0x080112d0                voicegroup054
                0x0803f6e0                voicegroup391
                0x0803b474                voicegroup379
                0x08042bfc                voicegroup405
                0x080459a8                song_table
 .rodata        0x08046cbc      0x6a4 glockens_c5.o
                0x08046cbc                glockens_c5
 .rodata        0x08047360      0x7f8 porgan_c4.o
                0x08047360                porgan_c4
 .rodata        0x08047b58      0xbcc acobs_c1.o
                0x08047b58                acobs_c1
 .rodata        0x08048724      0xf38 slapbs_c1.o
                0x08048724                slapbs_c1
 .rodata        0x0804965c      0xc74 synbs_c2.o
                0x0804965c                synbs_c2
 .rodata        0x0804a2d0     0x14d0 timpani_c2.o
                0x0804a2d0                timpani_c2
 .rodata        0x0804b7a0     0x16b0 octcho_c3.o
                0x0804b7a0                octcho_c3
 .rodata        0x0804ce50     0x1344 oboe_c3.o
                0x0804ce50                oboe_c3
 .rodata        0x0804e194      0xaa4 oboe_c4.o
                0x0804e194                oboe_c4
 .rodata        0x0804ec38     0x1314 p_gt_c3.o
                0x0804ec38                p_gt_c3
 .rodata        0x0804ff4c     0x35fc slapb_c1.o
                0x0804ff4c                slapb_c1
 .rodata        0x08053548      0x4d8 vosne.o
                0x08053548                vosne
 .rodata        0x08053a20     0x18dc woodat1.o
                0x08053a20                woodat1
 .rodata        0x080552fc     0x1328 woodat2.o
                0x080552fc                woodat2
 .rodata        0x08056624      0x4a0 bdrum.o
                0x08056624                bdrum
 .rodata        0x08056ac4      0x6f4 snare_l.o
                0x08056ac4                snare_l
 .rodata        0x080571b8      0x890 hand_clap.o
                0x080571b8                hand_clap
 .rodata        0x08057a48      0x878 oce_snare.o
                0x08057a48                oce_snare
 .rodata        0x080582c0     0x1040 tom.o
                0x080582c0                tom
 .rodata        0x08059300      0x414 closehh.o
                0x08059300                closehh
 .rodata        0x08059714      0xe30 openhh.o
                0x08059714                openhh
 .rodata        0x0805a544      0xf94 ride.o
                0x0805a544                ride
 .rodata        0x0805b4d8      0x8b4 tambo.o
                0x0805b4d8                tambo
 .rodata        0x0805bd8c      0x8e4 splash.o
                0x0805bd8c                splash
 .rodata        0x0805c670      0xf2c cymbal.o
                0x0805c670                cymbal
 .rodata        0x0805d59c      0x518 h_conga.o
                0x0805d59c                h_conga
 .rodata        0x0805dab4      0x5c8 l_conga.o
                0x0805dab4                l_conga
 .rodata        0x0805e07c      0xf18 ti_bass.o
                0x0805e07c                ti_bass
 .rodata        0x0805ef94     0x1974 rimshot.o
                0x0805ef94                rimshot
 .rodata        0x08060908     0x20dc tom1.o
                0x08060908                tom1
 .rodata        0x080629e4     0x7830 ridecap.o
                0x080629e4                ridecap
 .rodata        0x0806a214      0x9b8 cowbell.o
                0x0806a214                cowbell
 .rodata        0x0806abcc      0xe80 indian.o
                0x0806abcc                indian
 .rodata        0x0806ba4c      0xe74 triyang.o
                0x0806ba4c                triyang
 .rodata        0x0806c8c0     0x1814 suzu.o
                0x0806c8c0                suzu
 .rodata        0x0806e0d4     0x15a4 kane.o
                0x0806e0d4                kane
 .rodata        0x0806f678     0x15e4 taiko.o
                0x0806f678                taiko
 .rodata        0x08070c5c     0x10f4 tsutsumi.o
                0x08070c5c                tsutsumi
 .rodata        0x08071d50      0xf60 piano1_c2.o
                0x08071d50                piano1_c2
 .rodata        0x08072cb0     0x1660 piano1_c3.o
                0x08072cb0                piano1_c3
 .rodata        0x08074310     0x155c piano1_c4.o
                0x08074310                piano1_c4
 .rodata        0x0807586c      0xb8c piano1_c6.o
                0x0807586c                piano1_c6
 .rodata        0x080763f8     0x35a4 str_c3.o
                0x080763f8                str_c3
 .rodata        0x0807999c     0x231c str_c4.o
                0x0807999c                str_c4
 .rodata        0x0807bcb8     0x36cc str_c5.o
                0x0807bcb8                str_c5
 .rodata        0x0807f384     0x1350 tr_c3.o
                0x0807f384                tr_c3
 .rodata        0x080806d4     0x1510 tr_c4.o
                0x080806d4                tr_c4
 .rodata        0x08081be4     0x1420 tr_c5.o
                0x08081be4                tr_c5
 .rodata        0x08083004     0x109c tuba_c1.o
                0x08083004                tuba_c1
 .rodata        0x080840a0     0x105c tuba_c2.o
                0x080840a0                tuba_c2
 .rodata        0x080850fc     0x6f94 horn_c3.o
                0x080850fc                horn_c3
 .rodata        0x0808c090     0x4584 horn_c4.o
                0x0808c090                horn_c4
 .rodata        0x08090614      0x764 flute_c5.o
                0x08090614                flute_c5
 .rodata        0x08090d78     0x1c50 ebase_c1.o
                0x08090d78                ebase_c1
 .rodata        0x080929c8     0x1804 koto_c4.o
                0x080929c8                koto_c4
 .rodata        0x080941cc     0x3bb8 shakuhachi_c4.o
                0x080941cc                shakuhachi_c4
 .rodata        0x08097d84     0x2238 koto_c3.o
                0x08097d84                koto_c3
 .rodata        0x08099fbc     0x1e70 ovgt_c3.o
                0x08099fbc                ovgt_c3
 .rodata        0x0809be2c     0x2ff0 disgt_c3.o
                0x0809be2c                disgt_c3
 .rodata        0x0809ee1c     0x2c54 disgt_c2.o
                0x0809ee1c                disgt_c2
 .rodata        0x080a1a70     0x4580 gamelam_c3.o
                0x080a1a70                gamelam_c3
 .rodata        0x080a5ff0     0x2948 pipeorg1_c3.o
                0x080a5ff0                pipeorg1_c3
 .rodata        0x080a8938     0x1760 pipeorg2_c4.o
                0x080a8938                pipeorg2_c4
 .rodata        0x080aa098     0x1644 voice_huu1.o
                0x080aa098                voice_huu1
 .rodata        0x080ab6dc     0x24a8 voice_haa1.o
                0x080ab6dc                voice_haa1
 .rodata        0x080adb84     0x2668 elep4_c3.o
                0x080adb84                elep4_c3
 .rodata        0x080b01ec     0x13a8 elep4_c4.o
                0x080b01ec                elep4_c4
 .rodata        0x080b1594     0x14d0 tim_sn_c2.o
                0x080b1594                tim_sn_c2
 .rodata        0x080b2a64      0xa0c ban.o
                0x080b2a64                ban
 .rodata        0x080b3470     0x1c14 psg_plus_c4.o
                0x080b3470                psg_plus_c4
 .rodata        0x080b5084     0x1960 bic_bell.o
                0x080b5084                bic_bell
 .rodata        0x080b69e4     0x14c4 door.o
                0x080b69e4                door
 .rodata        0x080b7ea8      0x73c pizz_c4.o
                0x080b7ea8                pizz_c4
 .rodata        0x080b85e4     0x1bf0 track.o
                0x080b85e4                track
 .rodata        0x080ba1d4     0x13b4 moter.o
                0x080ba1d4                moter
 .rodata        0x080bb588     0x2684 kaminari.o
                0x080bb588                kaminari
 .rodata        0x080bdc0c     0x1244 kaze.o
                0x080bdc0c                kaze
 .rodata        0x080bee50     0x1010 bubble.o
                0x080bee50                bubble
 .rodata        0x080bfe60     0x1308 iwa.o
                0x080bfe60                iwa
 .rodata        0x080c1168     0x210c fire.o
                0x080c1168                fire
 .rodata        0x080c3274     0x1fdc megab_c4.o
                0x080c3274                megab_c4
 .rodata        0x080c5250     0x2210 nami.o
                0x080c5250                nami
 .rodata        0x080c7460      0x7cc gigigi.o
                0x080c7460                gigigi
 .rodata        0x080c7c2c     0x1970 tu_bells_c4.o
                0x080c7c2c                tu_bells_c4
 .rodata        0x080c959c     0x1fb0 bomb.o
                0x080c959c                bomb
 .rodata        0x080cb54c     0x32e0 big_bone_c2.o
                0x080cb54c                big_bone_c2
 .rodata        0x080ce82c      0xa30 harp_c5.o
                0x080ce82c                harp_c5
 .rodata        0x080cf25c      0xa34 xylophone_c5.o
                0x080cf25c                xylophone_c5
 .rodata        0x080cfc90     0x1b40 kansei.o
                0x080cfc90                kansei
 .rodata        0x080d17d0      0x8c8 tamakoro.o
                0x080d17d0                tamakoro
 .rodata        0x080d2098     0x13d0 accord_c4.o
                0x080d2098                accord_c4
 .rodata        0x080d3468      0xc10 voice_a.o
                0x080d3468                voice_a
 .rodata        0x080d4078      0xb90 voice_i.o
                0x080d4078                voice_i
 .rodata        0x080d4c08      0xa9c voice_u.o
                0x080d4c08                voice_u
 .rodata        0x080d56a4      0x948 voice_e.o
                0x080d56a4                voice_e
 .rodata        0x080d5fec      0xa48 voice_o.o
                0x080d5fec                voice_o
 .rodata        0x080d6a34      0xc88 voice_n.o
                0x080d6a34                voice_n
 .rodata        0x080d76bc     0x108c pv001.o
                0x080d76bc                pv001
 .rodata        0x080d8748     0x1090 pv002.o
                0x080d8748                pv002
 .rodata        0x080d97d8     0x1358 pv003.o
                0x080d97d8                pv003
 .rodata        0x080dab30      0xe70 pv004.o
                0x080dab30                pv004
 .rodata        0x080db9a0      0xe80 pv005.o
                0x080db9a0                pv005
 .rodata        0x080dc820     0x1348 pv006.o
                0x080dc820                pv006
 .rodata        0x080ddb68      0xe74 pv007.o
                0x080ddb68                pv007
 .rodata        0x080de9dc     0x1140 pv008.o
                0x080de9dc                pv008
 .rodata        0x080dfb1c     0x1348 pv009.o
                0x080dfb1c                pv009
 .rodata        0x080e0e64      0x858 pv010.o
                0x080e0e64                pv010
 .rodata        0x080e16bc     0x1750 pv011.o
                0x080e16bc                pv011
 .rodata        0x080e2e0c      0xa08 pv012.o
                0x080e2e0c                pv012
 .rodata        0x080e3814     0x1044 pv013.o
                0x080e3814                pv013
 .rodata        0x080e4858     0x123c pv014.o
                0x080e4858                pv014
 .rodata        0x080e5a94     0x135c pv015.o
                0x080e5a94                pv015
 .rodata        0x080e6df0      0x3e8 pv016.o
                0x080e6df0                pv016
 .rodata        0x080e71d8      0xf08 pv017.o
                0x080e71d8                pv017
 .rodata        0x080e80e0     0x1134 pv018.o
                0x080e80e0                pv018
 .rodata        0x080e9214      0x7e0 pv019.o
                0x080e9214                pv019
 .rodata        0x080e99f4      0x984 pv020.o
                0x080e99f4                pv020
 .rodata        0x080ea378     0x11a4 pv021.o
                0x080ea378                pv021
 .rodata        0x080eb51c     0x113c pv022.o
                0x080eb51c                pv022
 .rodata        0x080ec658     0x134c pv023.o
                0x080ec658                pv023
 .rodata        0x080ed9a4     0x1358 pv024.o
                0x080ed9a4                pv024
 .rodata        0x080eecfc     0x10a8 pv025.o
                0x080eecfc                pv025
 .rodata        0x080efda4     0x17c0 pv026.o
                0x080efda4                pv026
 .rodata        0x080f1564      0x954 pv027.o
                0x080f1564                pv027
 .rodata        0x080f1eb8      0xd90 pv028.o
                0x080f1eb8                pv028
 .rodata        0x080f2c48      0x9b0 pv029.o
                0x080f2c48                pv029
 .rodata        0x080f35f8      0xcc8 pv030.o
                0x080f35f8                pv030
 .rodata        0x080f42c0     0x10e0 pv031.o
                0x080f42c0                pv031
 .rodata        0x080f53a0      0xa68 pv032.o
                0x080f53a0                pv032
 .rodata        0x080f5e08      0xc14 pv033.o
                0x080f5e08                pv033
 .rodata        0x080f6a1c     0x186c pv034.o
                0x080f6a1c                pv034
 .rodata        0x080f8288      0x870 pv035.o
                0x080f8288                pv035
 .rodata        0x080f8af8      0xa90 pv036.o
                0x080f8af8                pv036
 .rodata        0x080f9588     0x17d0 pv037.o
                0x080f9588                pv037
 .rodata        0x080fad58     0x186c pv038.o
                0x080fad58                pv038
 .rodata        0x080fc5c4      0x564 pv039.o
                0x080fc5c4                pv039
 .rodata        0x080fcb28      0x6c8 pv040.o
                0x080fcb28                pv040
 .rodata        0x080fd1f0     0x136c pv041.o
                0x080fd1f0                pv041
 .rodata        0x080fe55c     0x1364 pv042.o
                0x080fe55c                pv042
 .rodata        0x080ff8c0      0xe9c pv043.o
                0x080ff8c0                pv043
 .rodata        0x0810075c      0xc7c pv044.o
                0x0810075c                pv044
 .rodata        0x081013d8     0x199c pv045.o
                0x081013d8                pv045
 .rodata        0x08102d74     0x1bf4 pv046.o
                0x08102d74                pv046
 .rodata        0x08104968     0x1e68 pv047.o
                0x08104968                pv047
 .rodata        0x081067d0      0xf80 pv048.o
                0x081067d0                pv048
 .rodata        0x08107750     0x1004 pv049.o
                0x08107750                pv049
 .rodata        0x08108754     0x1370 pv050.o
                0x08108754                pv050
 .rodata        0x08109ac4     0x136c pv051.o
                0x08109ac4                pv051
 .rodata        0x0810ae30      0x990 pv052.o
                0x0810ae30                pv052
 .rodata        0x0810b7c0     0x12dc pv053.o
                0x0810b7c0                pv053
 .rodata        0x0810ca9c      0xd28 pv054.o
                0x0810ca9c                pv054
 .rodata        0x0810d7c4      0xb48 pv055.o
                0x0810d7c4                pv055
 .rodata        0x0810e30c     0x1060 pv056.o
                0x0810e30c                pv056
 .rodata        0x0810f36c     0x1030 pv057.o
                0x0810f36c                pv057
 .rodata        0x0811039c      0xd64 pv058.o
                0x0811039c                pv058
 .rodata        0x08111100     0x113c pv059.o
                0x08111100                pv059
 .rodata        0x0811223c      0xb1c pv060.o
                0x0811223c                pv060
 .rodata        0x08112d58      0x6a8 pv061.o
                0x08112d58                pv061
 .rodata        0x08113400      0xb24 pv062.o
                0x08113400                pv062
 .rodata        0x08113f24     0x1764 pv063.o
                0x08113f24                pv063
 .rodata        0x08115688     0x1ae8 pv064.o
                0x08115688                pv064
 .rodata        0x08117170     0x1f9c pv065.o
                0x08117170                pv065
 .rodata        0x0811910c      0xd64 pv066.o
                0x0811910c                pv066
 .rodata        0x08119e70      0xd90 pv067.o
                0x08119e70                pv067
 .rodata        0x0811ac00     0x1088 pv068.o
                0x0811ac00                pv068
 .rodata        0x0811bc88      0x78c pv069.o
                0x0811bc88                pv069
 .rodata        0x0811c414      0xea0 pv070.o
                0x0811c414                pv070
 .rodata        0x0811d2b4     0x134c pv071.o
                0x0811d2b4                pv071
 .rodata        0x0811e600      0xff0 pv072.o
                0x0811e600                pv072
 .rodata        0x0811f5f0     0x16fc pv073.o
                0x0811f5f0                pv073
 .rodata        0x08120cec     0x17b4 pv074.o
                0x08120cec                pv074
 .rodata        0x081224a0     0x1be8 pv075.o
                0x081224a0                pv075
 .rodata        0x08124088      0xe2c pv076.o
                0x08124088                pv076
 .rodata        0x08124eb4      0xf10 pv077.o
                0x08124eb4                pv077
 .rodata        0x08125dc4     0x12a0 pv078.o
                0x08125dc4                pv078
 .rodata        0x08127064      0x768 pv079.o
                0x08127064                pv079
 .rodata        0x081277cc      0xd70 pv080.o
                0x081277cc                pv080
 .rodata        0x0812853c     0x1344 pv081.o
                0x0812853c                pv081
 .rodata        0x08129880     0x17e8 pv082.o
                0x08129880                pv082
 .rodata        0x0812b068      0x77c pv083.o
                0x0812b068                pv083
 .rodata        0x0812b7e4     0x1344 pv084.o
                0x0812b7e4                pv084
 .rodata        0x0812cb28     0x1378 pv085.o
                0x0812cb28                pv085
 .rodata        0x0812dea0     0x11f0 pv086.o
                0x0812dea0                pv086
 .rodata        0x0812f090     0x1524 pv087.o
                0x0812f090                pv087
 .rodata        0x081305b4      0xa88 pv088.o
                0x081305b4                pv088
 .rodata        0x0813103c      0xec0 pv089.o
                0x0813103c                pv089
 .rodata        0x08131efc      0xf74 pv090.o
                0x08131efc                pv090
 .rodata        0x08132e70     0x14c4 pv091.o
                0x08132e70                pv091
 .rodata        0x08134334     0x1750 pv092.o
                0x08134334                pv092
 .rodata        0x08135a84     0x1780 pv093.o
                0x08135a84                pv093
 .rodata        0x08137204      0xec0 pv094.o
                0x08137204                pv094
 .rodata        0x081380c4     0x18c4 pv095.o
                0x081380c4                pv095
 .rodata        0x08139988     0x1d18 pv096.o
                0x08139988                pv096
 .rodata        0x0813b6a0     0x1d04 pv097.o
                0x0813b6a0                pv097
 .rodata        0x0813d3a4     0x184c pv098.o
                0x0813d3a4                pv098
 .rodata        0x0813ebf0     0x1858 pv099.o
                0x0813ebf0                pv099
 .rodata        0x08140448     0x18c4 pv100.o
                0x08140448                pv100
 .rodata        0x08141d0c     0x1938 pv101.o
                0x08141d0c                pv101
 .rodata        0x08143644     0x12e0 pv102.o
                0x08143644                pv102
 .rodata        0x08144924     0x1fe4 pv103.o
                0x08144924                pv103
 .rodata        0x08146908      0xf20 pv104.o
                0x08146908                pv104
 .rodata        0x08147828      0xe70 pv105.o
                0x08147828                pv105
 .rodata        0x08148698     0x12ac pv106.o
                0x08148698                pv106
 .rodata        0x08149944     0x11d8 pv107.o
                0x08149944                pv107
 .rodata        0x0814ab1c      0xf28 pv108.o
                0x0814ab1c                pv108
 .rodata        0x0814ba44     0x145c pv109.o
                0x0814ba44                pv109
 .rodata        0x0814cea0     0x15ac pv110.o
                0x0814cea0                pv110
 .rodata        0x0814e44c     0x136c pv111.o
                0x0814e44c                pv111
 .rodata        0x0814f7b8     0x146c pv112.o
                0x0814f7b8                pv112
 .rodata        0x08150c24      0xecc pv113.o
                0x08150c24                pv113
 .rodata        0x08151af0      0xf1c pv114.o
                0x08151af0                pv114
 .rodata        0x08152a0c     0x12b4 pv115.o
                0x08152a0c                pv115
 .rodata        0x08153cc0      0x97c pv116.o
                0x08153cc0                pv116
 .rodata        0x0815463c      0x86c pv117.o
                0x0815463c                pv117
 .rodata        0x08154ea8      0x9d8 pv118.o
                0x08154ea8                pv118
 .rodata        0x08155880     0x1358 pv119.o
                0x08155880                pv119
 .rodata        0x08156bd8     0x13e8 pv120.o
                0x08156bd8                pv120
 .rodata        0x08157fc0     0x14dc pv121.o
                0x08157fc0                pv121
 .rodata        0x0815949c     0x12f0 pv122.o
                0x0815949c                pv122
 .rodata        0x0815a78c      0xd5c pv123.o
                0x0815a78c                pv123
 .rodata        0x0815b4e8     0x2f74 pv124.o
                0x0815b4e8                pv124
 .rodata        0x0815e45c     0x1ee4 pv125.o
                0x0815e45c                pv125
 .rodata        0x08160340      0xf7c pv126.o
                0x08160340                pv126
 .rodata        0x081612bc      0xc5c pv127.o
                0x081612bc                pv127
 .rodata        0x08161f18     0x1254 pv128.o
                0x08161f18                pv128
 .rodata        0x0816316c     0x1308 pv129.o
                0x0816316c                pv129
 .rodata        0x08164474     0x1434 pv130.o
                0x08164474                pv130
 .rodata        0x081658a8      0xed4 pv131.o
                0x081658a8                pv131
 .rodata        0x0816677c      0xb1c pv132.o
                0x0816677c                pv132
 .rodata        0x08167298      0xe38 pv133.o
                0x08167298                pv133
 .rodata        0x081680d0     0x1618 pv134.o
                0x081680d0                pv134
 .rodata        0x081696e8      0xfd4 pv135.o
                0x081696e8                pv135
 .rodata        0x0816a6bc      0xf84 pv136.o
                0x0816a6bc                pv136
 .rodata        0x0816b640     0x140c pv137.o
                0x0816b640                pv137
 .rodata        0x0816ca4c      0xd58 pv138.o
                0x0816ca4c                pv138
 .rodata        0x0816d7a4      0xd54 pv139.o
                0x0816d7a4                pv139
 .rodata        0x0816e4f8      0xc54 pv140.o
                0x0816e4f8                pv140
 .rodata        0x0816f14c      0xdbc pv141.o
                0x0816f14c                pv141
 .rodata        0x0816ff08     0x185c pv142.o
                0x0816ff08                pv142
 .rodata        0x08171764      0x53c pv143.o
                0x08171764                pv143
 .rodata        0x08171ca0     0x17a8 pv144.o
                0x08171ca0                pv144
 .rodata        0x08173448      0xf78 pv145.o
                0x08173448                pv145
 .rodata        0x081743c0     0x17ac pv146.o
                0x081743c0                pv146
 .rodata        0x08175b6c      0xb9c pv147.o
                0x08175b6c                pv147
 .rodata        0x08176708     0x10a8 pv148.o
                0x08176708                pv148
 .rodata        0x081777b0     0x130c pv149.o
                0x081777b0                pv149
 .rodata        0x08178abc     0x1e68 pv150.o
                0x08178abc                pv150
 .rodata        0x0817a924     0x1e68 pv151.o
                0x0817a924                pv151
 .rodata        0x0817c78c      0x540 pv152.o
                0x0817c78c                pv152
 .rodata        0x0817cccc      0x8cc pv153.o
                0x0817cccc                pv153
 .rodata        0x0817d598     0x1038 pv154.o
                0x0817d598                pv154
 .rodata        0x0817e5d0      0x704 pv155.o
                0x0817e5d0                pv155
 .rodata        0x0817ecd4      0xbe8 pv156.o
                0x0817ecd4                pv156
 .rodata        0x0817f8bc     0x2610 pv157.o
                0x0817f8bc                pv157
 .rodata        0x08181ecc     0x1258 pv158.o
                0x08181ecc                pv158
 .rodata        0x08183124     0x143c pv159.o
                0x08183124                pv159
 .rodata        0x08184560     0x1984 pv160.o
                0x08184560                pv160
 .rodata        0x08185ee4      0x428 pv161.o
                0x08185ee4                pv161
 .rodata        0x0818630c      0x648 pv162.o
                0x0818630c                pv162
 .rodata        0x08186954      0xae4 pv163.o
                0x08186954                pv163
 .rodata        0x08187438     0x1530 pv164.o
                0x08187438                pv164
 .rodata        0x08188968      0x6f8 pv165.o
                0x08188968                pv165
 .rodata        0x08189060      0x864 pv166.o
                0x08189060                pv166
 .rodata        0x081898c4      0xd64 pv167.o
                0x081898c4                pv167
 .rodata        0x0818a628      0xc54 pv168.o
                0x0818a628                pv168
 .rodata        0x0818b27c     0x1730 pv169.o
                0x0818b27c                pv169
 .rodata        0x0818c9ac      0xcb0 pv170.o
                0x0818c9ac                pv170
 .rodata        0x0818d65c      0xa8c pv171.o
                0x0818d65c                pv171
 .rodata        0x0818e0e8      0x754 pv172.o
                0x0818e0e8                pv172
 .rodata        0x0818e83c      0x5f0 pv173.o
                0x0818e83c                pv173
 .rodata        0x0818ee2c      0x6fc pv174.o
                0x0818ee2c                pv174
 .rodata        0x0818f528      0xae8 pv175.o
                0x0818f528                pv175
 .rodata        0x08190010      0x700 pv176.o
                0x08190010                pv176
 .rodata        0x08190710      0xa90 pv177.o
                0x08190710                pv177
 .rodata        0x081911a0      0xecc pv178.o
                0x081911a0                pv178
 .rodata        0x0819206c      0x758 pv179.o
                0x0819206c                pv179
 .rodata        0x081927c4      0xdb4 pv180.o
                0x081927c4                pv180
 .rodata        0x08193578     0x1080 pv181.o
                0x08193578                pv181
 .rodata        0x081945f8      0xe18 pv182.o
                0x081945f8                pv182
 .rodata        0x08195410      0xd14 pv183.o
                0x08195410                pv183
 .rodata        0x08196124     0x10ec pv184.o
                0x08196124                pv184
 .rodata        0x08197210     0x1030 pv185.o
                0x08197210                pv185
 .rodata        0x08198240     0x1244 pv186.o
                0x08198240                pv186
 .rodata        0x08199484      0x86c pv187.o
                0x08199484                pv187
 .rodata        0x08199cf0      0xd08 pv188.o
                0x08199cf0                pv188
 .rodata        0x0819a9f8     0x103c pv189.o
                0x0819a9f8                pv189
 .rodata        0x0819ba34      0xe20 pv190.o
                0x0819ba34                pv190
 .rodata        0x0819c854      0x814 pv191.o
                0x0819c854                pv191
 .rodata        0x0819d068      0xfe0 pv192.o
                0x0819d068                pv192
 .rodata        0x0819e048     0x1108 pv193.o
                0x0819e048                pv193
 .rodata        0x0819f150      0x760 pv194.o
                0x0819f150                pv194
 .rodata        0x0819f8b0      0xd60 pv195.o
                0x0819f8b0                pv195
 .rodata        0x081a0610     0x13b4 pv196.o
                0x081a0610                pv196
 .rodata        0x081a19c4      0xf80 pv197.o
                0x081a19c4                pv197
 .rodata        0x081a2944     0x10c4 pv198.o
                0x081a2944                pv198
 .rodata        0x081a3a08     0x17e4 pv199.o
                0x081a3a08                pv199
 .rodata        0x081a51ec      0xba0 pv200.o
                0x081a51ec                pv200
 .rodata        0x081a5d8c      0xd28 pv201.o
                0x081a5d8c                pv201
 .rodata        0x081a6ab4     0x149c pv202.o
                0x081a6ab4                pv202
 .rodata        0x081a7f50      0xeb4 pv203.o
                0x081a7f50                pv203
 .rodata        0x081a8e04      0xd60 pv204.o
                0x081a8e04                pv204
 .rodata        0x081a9b64     0x1408 pv205.o
                0x081a9b64                pv205
 .rodata        0x081aaf6c      0xfe0 pv206.o
                0x081aaf6c                pv206
 .rodata        0x081abf4c      0xc20 pv207.o
                0x081abf4c                pv207
 .rodata        0x081acb6c     0x2628 pv208.o
                0x081acb6c                pv208
 .rodata        0x081af194      0xe74 pv209.o
                0x081af194                pv209
 .rodata        0x081b0008     0x17a4 pv210.o
                0x081b0008                pv210
 .rodata        0x081b17ac      0xb9c pv211.o
                0x081b17ac                pv211
 .rodata        0x081b2348     0x16fc pv212.o
                0x081b2348                pv212
 .rodata        0x081b3a44      0xa34 pv213.o
                0x081b3a44                pv213
 .rodata        0x081b4478     0x1254 pv214.o
                0x081b4478                pv214
 .rodata        0x081b56cc      0x924 pv215.o
                0x081b56cc                pv215
 .rodata        0x081b5ff0     0x108c pv216.o
                0x081b5ff0                pv216
 .rodata        0x081b707c     0x1dd8 pv217.o
                0x081b707c                pv217
 .rodata        0x081b8e54     0x1118 pv218.o
                0x081b8e54                pv218
 .rodata        0x081b9f6c     0x1508 pv219.o
                0x081b9f6c                pv219
 .rodata        0x081bb474      0xca8 pv220.o
                0x081bb474                pv220
 .rodata        0x081bc11c      0xcf4 pv221.o
                0x081bc11c                pv221
 .rodata        0x081bce10      0xce0 pv222.o
                0x081bce10                pv222
 .rodata        0x081bdaf0      0xa90 pv223.o
                0x081bdaf0                pv223
 .rodata        0x081be580     0x1a44 pv224.o
                0x081be580                pv224
 .rodata        0x081bffc4     0x1034 pv225.o
                0x081bffc4                pv225
 .rodata        0x081c0ff8      0xfc8 pv226.o
                0x081c0ff8                pv226
 .rodata        0x081c1fc0     0x1808 pv227.o
                0x081c1fc0                pv227
 .rodata        0x081c37c8      0xca8 pv228.o
                0x081c37c8                pv228
 .rodata        0x081c4470     0x13b0 pv229.o
                0x081c4470                pv229
 .rodata        0x081c5820      0xdd8 pv230.o
                0x081c5820                pv230
 .rodata        0x081c65f8      0xb50 pv231.o
                0x081c65f8                pv231
 .rodata        0x081c7148     0x1124 pv232.o
                0x081c7148                pv232
 .rodata        0x081c826c      0xfb8 pv233.o
                0x081c826c                pv233
 .rodata        0x081c9224     0x167c pv234.o
                0x081c9224                pv234
 .rodata        0x081ca8a0      0xa34 pv235.o
                0x081ca8a0                pv235
 .rodata        0x081cb2d4     0x1028 pv236.o
                0x081cb2d4                pv236
 .rodata        0x081cc2fc      0xde0 pv237.o
                0x081cc2fc                pv237
 .rodata        0x081cd0dc      0xbb4 pv238.o
                0x081cd0dc                pv238
 .rodata        0x081cdc90      0xa8c pv239.o
                0x081cdc90                pv239
 .rodata        0x081ce71c      0xe70 pv240.o
                0x081ce71c                pv240
 .rodata        0x081cf58c      0xedc pv241.o
                0x081cf58c                pv241
 .rodata        0x081d0468     0x1094 pv242.o
                0x081d0468                pv242
 .rodata        0x081d14fc     0x1170 pv243.o
                0x081d14fc                pv243
 .rodata        0x081d266c     0x1474 pv244.o
                0x081d266c                pv244
 .rodata        0x081d3ae0     0x1248 pv245.o
                0x081d3ae0                pv245
 .rodata        0x081d4d28      0xcb0 pv246.o
                0x081d4d28                pv246
 .rodata        0x081d59d8      0x870 pv247.o
                0x081d59d8                pv247
 .rodata        0x081d6248     0x1760 pv248.o
                0x081d6248                pv248
 .rodata        0x081d79a8     0x25f8 pv249.o
                0x081d79a8                pv249
 .rodata        0x081d9fa0     0x1694 pv250.o
                0x081d9fa0                pv250
 .rodata        0x081db634      0xe78 pv251.o
                0x081db634                pv251
 .rodata        0x081dc4ac      0x860 pv252.o
                0x081dc4ac                pv252
 .rodata        0x081dcd0c      0xac0 pv253.o
                0x081dcd0c                pv253
 .rodata        0x081dd7cc      0x94c pv254.o
                0x081dd7cc                pv254
 .rodata        0x081de118      0xc5c pv255.o
                0x081de118                pv255
 .rodata        0x081ded74     0x1508 pv256.o
                0x081ded74                pv256
 .rodata        0x081e027c      0xa98 pv257.o
                0x081e027c                pv257
 .rodata        0x081e0d14      0xc30 pv258.o
                0x081e0d14                pv258
 .rodata        0x081e1944      0xde0 pv259.o
                0x081e1944                pv259
 .rodata        0x081e2724      0xba0 pv260.o
                0x081e2724                pv260
 .rodata        0x081e32c4     0x170c pv261.o
                0x081e32c4                pv261
 .rodata        0x081e49d0      0x988 pv262.o
                0x081e49d0                pv262
 .rodata        0x081e5358      0xa68 pv263.o
                0x081e5358                pv263
 .rodata        0x081e5dc0      0x598 pv264.o
                0x081e5dc0                pv264
 .rodata        0x081e6358      0xb1c pv265.o
                0x081e6358                pv265
 .rodata        0x081e6e74      0x954 pv266.o
                0x081e6e74                pv266
 .rodata        0x081e77c8      0x600 pv267.o
                0x081e77c8                pv267
 .rodata        0x081e7dc8      0x904 pv268.o
                0x081e7dc8                pv268
 .rodata        0x081e86cc     0x11b0 pv269.o
                0x081e86cc                pv269
 .rodata        0x081e987c      0xc6c pv270.o
                0x081e987c                pv270
 .rodata        0x081ea4e8      0x9a8 pv271.o
                0x081ea4e8                pv271
 .rodata        0x081eae90     0x1cd4 pv272.o
                0x081eae90                pv272
 .rodata        0x081ecb64     0x1f80 pv273.o
                0x081ecb64                pv273
 .rodata        0x081eeae4      0xba8 pv274.o
                0x081eeae4                pv274
 .rodata        0x081ef68c     0x1474 pv275.o
                0x081ef68c                pv275
 .rodata        0x081f0b00     0x1a1c pv276.o
                0x081f0b00                pv276
 .rodata        0x081f251c      0x784 pv277.o
                0x081f251c                pv277
 .rodata        0x081f2ca0     0x1104 pv278.o
                0x081f2ca0                pv278
 .rodata        0x081f3da4     0x1680 pv279.o
                0x081f3da4                pv279
 .rodata        0x081f5424      0xbc8 pv280.o
                0x081f5424                pv280
 .rodata        0x081f5fec      0xc40 pv281.o
                0x081f5fec                pv281
 .rodata        0x081f6c2c      0xca8 pv282.o
                0x081f6c2c                pv282
 .rodata        0x081f78d4      0x840 pv283.o
                0x081f78d4                pv283
 .rodata        0x081f8114      0x468 pv284.o
                0x081f8114                pv284
 .rodata        0x081f857c      0xe94 pv285.o
                0x081f857c                pv285
 .rodata        0x081f9410     0x10d0 pv286.o
                0x081f9410                pv286
 .rodata        0x081fa4e0      0x82c pv287.o
                0x081fa4e0                pv287
 .rodata        0x081fad0c      0xb68 pv288.o
                0x081fad0c                pv288
 .rodata        0x081fb874     0x13c4 pv289.o
                0x081fb874                pv289
 .rodata        0x081fcc38      0xa14 pv290.o
                0x081fcc38                pv290
 .rodata        0x081fd64c      0x8cc pv291.o
                0x081fd64c                pv291
 .rodata        0x081fdf18     0x102c pv292.o
                0x081fdf18                pv292
 .rodata        0x081fef44      0x838 pv293.o
                0x081fef44                pv293
 .rodata        0x081ff77c     0x1044 pv294.o
                0x081ff77c                pv294
 .rodata        0x082007c0      0xcac pv295.o
                0x082007c0                pv295
 .rodata        0x0820146c      0xa1c pv296.o
                0x0820146c                pv296
 .rodata        0x08201e88      0xc30 pv297.o
                0x08201e88                pv297
 .rodata        0x08202ab8     0x1864 pv298.o
                0x08202ab8                pv298
 .rodata        0x0820431c      0x884 pv299.o
                0x0820431c                pv299
 .rodata        0x08204ba0      0xe58 pv300.o
                0x08204ba0                pv300
 .rodata        0x082059f8      0x9ec pv301.o
                0x082059f8                pv301
 .rodata        0x082063e4      0x670 pv302.o
                0x082063e4                pv302
 .rodata        0x08206a54      0xc28 pv303.o
                0x08206a54                pv303
 .rodata        0x0820767c      0x7b8 pv304.o
                0x0820767c                pv304
 .rodata        0x08207e34      0x75c pv305.o
                0x08207e34                pv305
 .rodata        0x08208590     0x10b8 pv306.o
                0x08208590                pv306
 .rodata        0x08209648      0xd64 pv307.o
                0x08209648                pv307
 .rodata        0x0820a3ac     0x14e4 pv308.o
                0x0820a3ac                pv308
 .rodata        0x0820b890      0x8fc pv309.o
                0x0820b890                pv309
 .rodata        0x0820c18c     0x1008 pv310.o
                0x0820c18c                pv310
 .rodata        0x0820d194      0xa80 pv311.o
                0x0820d194                pv311
 .rodata        0x0820dc14     0x13b4 pv312.o
                0x0820dc14                pv312
 .rodata        0x0820efc8      0x714 pv313.o
                0x0820efc8                pv313
 .rodata        0x0820f6dc     0x1518 pv314.o
                0x0820f6dc                pv314
 .rodata        0x08210bf4      0x804 pv315.o
                0x08210bf4                pv315
 .rodata        0x082113f8     0x1160 pv316.o
                0x082113f8                pv316
 .rodata        0x08212558      0x94c pv317.o
                0x08212558                pv317
 .rodata        0x08212ea4     0x1720 pv318.o
                0x08212ea4                pv318
 .rodata        0x082145c4      0x93c pv319.o
                0x082145c4                pv319
 .rodata        0x08214f00     0x10fc pv320.o
                0x08214f00                pv320
 .rodata        0x08215ffc      0xc04 pv321.o
                0x08215ffc                pv321
 .rodata        0x08216c00     0x18b8 pv322.o
                0x08216c00                pv322
 .rodata        0x082184b8      0x740 pv323.o
                0x082184b8                pv323
 .rodata        0x08218bf8      0xca0 pv324.o
                0x08218bf8                pv324
 .rodata        0x08219898      0xa24 pv325.o
                0x08219898                pv325
 .rodata        0x0821a2bc      0xe04 pv326.o
                0x0821a2bc                pv326
 .rodata        0x0821b0c0     0x1a08 pv327.o
                0x0821b0c0                pv327
 .rodata        0x0821cac8      0x8f0 pv328.o
                0x0821cac8                pv328
 .rodata        0x0821d3b8     0x16b0 pv329.o
                0x0821d3b8                pv329
 .rodata        0x0821ea68      0xc84 pv330.o
                0x0821ea68                pv330
 .rodata        0x0821f6ec     0x1360 pv331.o
                0x0821f6ec                pv331
 .rodata        0x08220a4c     0x17fc pv332.o
                0x08220a4c                pv332
 .rodata        0x08222248     0x102c pv333.o
                0x08222248                pv333
 .rodata        0x08223274      0x7d4 pv334.o
                0x08223274                pv334
 .rodata        0x08223a48     0x2744 pv335.o
                0x08223a48                pv335
 .rodata        0x0822618c      0xa7c pv336.o
                0x0822618c                pv336
 .rodata        0x08226c08      0x820 pv337.o
                0x08226c08                pv337
 .rodata        0x08227428     0x1084 pv338.o
                0x08227428                pv338
 .rodata        0x082284ac      0x5b4 pv339.o
                0x082284ac                pv339
 .rodata        0x08228a60      0xbd8 pv340.o
                0x08228a60                pv340
 .rodata        0x08229638     0x244c pv341.o
                0x08229638                pv341
 .rodata        0x0822ba84     0x1250 pv342.o
                0x0822ba84                pv342
 .rodata        0x0822ccd4      0xfe8 pv343.o
                0x0822ccd4                pv343
 .rodata        0x0822dcbc     0x166c pv344.o
                0x0822dcbc                pv344
 .rodata        0x0822f328      0x9a8 pv345.o
                0x0822f328                pv345
 .rodata        0x0822fcd0     0x1d30 pv346.o
                0x0822fcd0                pv346
 .rodata        0x08231a00      0xbb8 pv347.o
                0x08231a00                pv347
 .rodata        0x082325b8     0x16d4 pv348.o
                0x082325b8                pv348
 .rodata        0x08233c8c      0x9a0 pv349.o
                0x08233c8c                pv349
 .rodata        0x0823462c     0x12d4 pv350.o
                0x0823462c                pv350
 .rodata        0x08235900     0x2778 pv351.o
                0x08235900                pv351
 .rodata        0x08238078      0x7d4 pv352.o
                0x08238078                pv352
 .rodata        0x0823884c     0x1408 pv353.o
                0x0823884c                pv353
 .rodata        0x08239c54     0x1fdc pv354.o
                0x08239c54                pv354
 .rodata        0x0823bc30     0x2000 pv355.o
                0x0823bc30                pv355
 .rodata        0x0823dc30     0x1704 pv356.o
                0x0823dc30                pv356
 .rodata        0x0823f334      0xc98 pv357.o
                0x0823f334                pv357
 .rodata        0x0823ffcc      0xb88 pv358.o
                0x0823ffcc                pv358
 .rodata        0x08240b54     0x1118 pv359.o
                0x08240b54                pv359
 .rodata        0x08241c6c      0x948 pv360.o
                0x08241c6c                pv360
 .rodata        0x082425b4     0x138c pv361.o
                0x082425b4                pv361
 .rodata        0x08243940      0xdb8 pv362.o
                0x08243940                pv362
 .rodata        0x082446f8      0xba4 pv363.o
                0x082446f8                pv363
 .rodata        0x0824529c      0xb80 pv364.o
                0x0824529c                pv364
 .rodata        0x08245e1c      0x92c pv365.o
                0x08245e1c                pv365
 .rodata        0x08246748     0x14d8 pv366.o
                0x08246748                pv366
 .rodata        0x08247c20     0x19a4 pv367.o
                0x08247c20                pv367
 .rodata        0x082495c4     0x1430 pv368.o
                0x082495c4                pv368
 .rodata        0x0824a9f4      0x4dc pv369.o
                0x0824a9f4                pv369
 .rodata        0x0824aed0     0x250c pv370.o
                0x0824aed0                pv370
 .rodata        0x0824d3dc     0x23b8 pv371.o
                0x0824d3dc                pv371
 .rodata        0x0824f794     0x1d2c pv372.o
                0x0824f794                pv372
 .rodata        0x082514c0     0x191c pv373.o
                0x082514c0                pv373
 .rodata        0x08252ddc      0xcc0 pv374.o
                0x08252ddc                pv374
 .rodata        0x08253a9c      0x8d8 pv375.o
                0x08253a9c                pv375
 .rodata        0x08254374     0x1e9c pv376.o
                0x08254374                pv376
 .rodata        0x08256210     0x20c4 pv377.o
                0x08256210                pv377
 .rodata        0x082582d4     0x1c60 pv378.o
                0x082582d4                pv378
 .rodata        0x08259f34      0xb90 pv379.o
                0x08259f34                pv379
 .rodata        0x0825aac4     0x1c48 pv380.o
                0x0825aac4                pv380
 .rodata        0x0825c70c      0xd28 pv381.o
                0x0825c70c                pv381
 .rodata        0x0825d434     0x2a10 pv382.o
                0x0825d434                pv382
 .rodata        0x0825fe44      0x824 pv383.o
                0x0825fe44                pv383
 .rodata        0x08260668     0x1108 pv384.o
                0x08260668                pv384
 .rodata        0x08261770     0x15f8 pv385.o
                0x08261770                pv385
 .rodata        0x08262d68      0xd84 pv386.o
                0x08262d68                pv386
 .rodata        0x08263aec     0x14d4 pv387.o
                0x08263aec                pv387
 .rodata        0x08264fc0      0xa10 pv388.o
                0x08264fc0                pv388
 .rodata        0x082659d0     0x1f60 shop.o
                0x082659d0                shop
 .rodata        0x08267930     0x1aa0 kiteki.o
                0x08267930                kiteki
 .rodata        0x082693d0     0x1f70 a_guitar_c4.o
                0x082693d0                a_guitar_c4
 .rodata        0x0826b340     0x1838 hau_c4.o
                0x0826b340                hau_c4
 .rodata        0x0826cb78      0x660 voice01_1.o
                0x0826cb78                voice01_1
 .rodata        0x0826d1d8      0x4e4 voice01_2.o
                0x0826d1d8                voice01_2
 .rodata        0x0826d6bc      0x950 voice01_3.o
                0x0826d6bc                voice01_3
 .rodata        0x0826e00c      0xa70 voice02_1.o
                0x0826e00c                voice02_1
 .rodata        0x0826ea7c      0x320 voice02_2.o
                0x0826ea7c                voice02_2
 .rodata        0x0826ed9c      0xc88 voice02_3.o
                0x0826ed9c                voice02_3
 .rodata        0x0826fa24      0x620 voice03_1.o
                0x0826fa24                voice03_1
 .rodata        0x08270044      0x388 voice03_2.o
                0x08270044                voice03_2
 .rodata        0x082703cc      0xde4 voice03_3.o
                0x082703cc                voice03_3
 .rodata        0x082711b0      0x970 voice04_1.o
                0x082711b0                voice04_1
 .rodata        0x08271b20      0x39c voice04_2.o
                0x08271b20                voice04_2
 .rodata        0x08271ebc      0x7b4 voice04_3.o
                0x08271ebc                voice04_3
 .rodata        0x08272670      0xd5c voice05_1.o
                0x08272670                voice05_1
 .rodata        0x082733cc      0x244 voice05_2.o
                0x082733cc                voice05_2
 .rodata        0x08273610      0xe40 voice05_3.o
                0x08273610                voice05_3
 .rodata        0x08274450      0x954 voice06_1.o
                0x08274450                voice06_1
 .rodata        0x08274da4      0x354 voice06_2.o
                0x08274da4                voice06_2
 .rodata        0x082750f8      0x634 voice06_3.o
                0x082750f8                voice06_3
 .rodata        0x0827572c      0xc6c voice07_1.o
                0x0827572c                voice07_1
 .rodata        0x08276398      0x598 voice07_2.o
                0x08276398                voice07_2
 .rodata        0x08276930      0xb04 voice07_3.o
                0x08276930                voice07_3
 .rodata        0x08277434      0x604 voice08_1.o
                0x08277434                voice08_1
 .rodata        0x08277a38      0x1f8 voice08_2.o
                0x08277a38                voice08_2
 .rodata        0x08277c30      0x964 voice08_3.o
                0x08277c30                voice08_3
 .rodata        0x08278594      0xf8c voice09_1.o
                0x08278594                voice09_1
 .rodata        0x08279520      0x638 voice09_2.o
                0x08279520                voice09_2
 .rodata        0x08279b58      0xad4 voice09_3.o
                0x08279b58                voice09_3
 .rodata        0x0827a62c      0xf44 voice10_1.o
                0x0827a62c                voice10_1
 .rodata        0x0827b570      0x578 voice10_2.o
                0x0827b570                voice10_2
 .rodata        0x0827bae8      0xe4c voice10_3.o
                0x0827bae8                voice10_3
 .rodata        0x0827c934      0xf08 voice11_1.o
                0x0827c934                voice11_1
 .rodata        0x0827d83c      0xad4 voice11_2.o
                0x0827d83c                voice11_2
 .rodata        0x0827e310      0xb94 voice11_3.o
                0x0827e310                voice11_3
 .rodata        0x0827eea4      0x9d8 voice12_1.o
                0x0827eea4                voice12_1
 .rodata        0x0827f87c      0x640 voice12_2.o
                0x0827f87c                voice12_2
 .rodata        0x0827febc      0xae0 voice12_3.o
                0x0827febc                voice12_3
 .rodata        0x0828099c      0x63c voice13_1.o
                0x0828099c                voice13_1
 .rodata        0x08280fd8      0x718 voice13_2.o
                0x08280fd8                voice13_2
 .rodata        0x082816f0      0x93c voice13_3.o
                0x082816f0                voice13_3
 .rodata        0x0828202c      0x7bc voice14_1.o
                0x0828202c                voice14_1
 .rodata        0x082827e8      0x564 voice14_2.o
                0x082827e8                voice14_2
 .rodata        0x08282d4c      0xd74 voice14_3.o
                0x08282d4c                voice14_3
 .rodata        0x08283ac0      0x47c voice15_1.o
                0x08283ac0                voice15_1
 .rodata        0x08283f3c      0x4ec voice15_2.o
                0x08283f3c                voice15_2
 .rodata        0x08284428      0x7c8 voice15_3.o
                0x08284428                voice15_3
 .rodata        0x08284bf0      0xbfc voice16_1.o
                0x08284bf0                voice16_1
 .rodata        0x082857ec      0x378 voice16_2.o
                0x082857ec                voice16_2
 .rodata        0x08285b64      0x7bc voice16_3.o
                0x08285b64                voice16_3
 .rodata        0x08286320      0xc64 voice17_1.o
                0x08286320                voice17_1
 .rodata        0x08286f84      0x4cc voice17_2.o
                0x08286f84                voice17_2
 .rodata        0x08287450      0xab0 voice17_3.o
                0x08287450                voice17_3
 .rodata        0x08287f00     0x13d0 test_c4.o
                0x08287f00                test_c4
 .rodata        0x082892d0     0x11c4 stpia_c3.o
                0x082892d0                stpia_c3
 .rodata        0x0828a494      0xa60 whis_c5.o
                0x0828a494                whis_c5
 .rodata        0x0828aef4     0x2100 fue1.o
                0x0828aef4                fue1
 .rodata        0x0828cff4        0x8 dummy.o
                0x0828cff4                dummy
 .rodata        0x0828cffc       0x24 se_kaifuku.o
                0x0828d014                se_kaifuku
 .rodata        0x0828d020       0x2c se_pc_login.o
                0x0828d040                se_pc_login
 .rodata        0x0828d04c       0x24 se_pc_off.o
                0x0828d064                se_pc_off
 .rodata        0x0828d070       0x44 se_pc_on.o
                0x0828d0a8                se_pc_on
 .rodata        0x0828d0b4       0x2c se_select.o
                0x0828d0d4                se_select
 .rodata        0x0828d0e0       0x1c se_win_open.o
                0x0828d0f0                se_win_open
 .rodata        0x0828d0fc       0x1c se_wall_hit.o
                0x0828d10c                se_wall_hit
 .rodata        0x0828d118       0x1c se_door.o
                0x0828d128                se_door
 .rodata        0x0828d134       0x34 se_kaidan.o
                0x0828d15c                se_kaidan
 .rodata        0x0828d168       0x24 se_dansa.o
                0x0828d180                se_dansa
 .rodata        0x0828d18c       0x1c se_jitensya.o
                0x0828d19c                se_jitensya
 .rodata        0x0828d1a8       0x30 se_kouka_l.o
                0x0828d1c8                se_kouka_l
 .rodata        0x0828d1d8       0x4c se_kouka_m.o
                0x0828d214                se_kouka_m
 .rodata        0x0828d224       0x7c se_kouka_h.o
                0x0828d290                se_kouka_h
 .rodata        0x0828d2a0       0x58 se_bowa2.o
                0x0828d2e4                se_bowa2
 .rodata        0x0828d2f8       0x54 se_poke_dead.o
                0x0828d338                se_poke_dead
 .rodata        0x0828d34c       0x48 se_nigeru.o
                0x0828d388                se_nigeru
 .rodata        0x0828d394       0x1c se_jido_doa.o
                0x0828d3a4                se_jido_doa
 .rodata        0x0828d3b0       0x54 se_naminori.o
                0x0828d3f8                se_naminori
 .rodata        0x0828d404       0x48 se_ban.o
                0x0828d440                se_ban
 .rodata        0x0828d44c       0x2c se_pin.o
                0x0828d46c                se_pin
 .rodata        0x0828d478       0x24 se_boo.o
                0x0828d490                se_boo
 .rodata        0x0828d49c       0x24 se_bowa.o
                0x0828d4b4                se_bowa
 .rodata        0x0828d4c0       0x90 se_jyuni.o
                0x0828d538                se_jyuni
 .rodata        0x0828d550       0x20 se_a.o
                0x0828d564                se_a
 .rodata        0x0828d570       0x20 se_i.o
                0x0828d584                se_i
 .rodata        0x0828d590       0x20 se_u.o
                0x0828d5a4                se_u
 .rodata        0x0828d5b0       0x20 se_e.o
                0x0828d5c4                se_e
 .rodata        0x0828d5d0       0x20 se_o.o
                0x0828d5e4                se_o
 .rodata        0x0828d5f0       0x20 se_n.o
                0x0828d604                se_n
 .rodata        0x0828d610       0x20 se_seikai.o
                0x0828d624                se_seikai
 .rodata        0x0828d630       0x30 se_hazure.o
                0x0828d654                se_hazure
 .rodata        0x0828d660      0x180 se_exp.o
                0x0828d7d4                se_exp
 .rodata        0x0828d7e0       0x24 se_jite_pyoko.o
                0x0828d7f8                se_jite_pyoko
 .rodata        0x0828d804       0x24 se_mu_pachi.o
                0x0828d81c                se_mu_pachi
 .rodata        0x0828d828       0x24 se_tk_kasya.o
                0x0828d840                se_tk_kasya
 .rodata        0x0828d84c       0x30 se_fu_zaku.o
                0x0828d870                se_fu_zaku
 .rodata        0x0828d87c       0x24 se_fu_zaku2.o
                0x0828d894                se_fu_zaku2
 .rodata        0x0828d8a0       0x4c se_fu_zuzuzu.o
                0x0828d8e0                se_fu_zuzuzu
 .rodata        0x0828d8ec       0x3c se_ru_gashin.o
                0x0828d918                se_ru_gashin
 .rodata        0x0828d928       0x54 se_ru_gasyan.o
                0x0828d96c                se_ru_gasyan
 .rodata        0x0828d97c       0x3c se_ru_bari.o
                0x0828d9a8                se_ru_bari
 .rodata        0x0828d9b8       0x54 se_ru_hyuu.o
                0x0828da00                se_ru_hyuu
 .rodata        0x0828da0c       0x48 se_ki_gasyan.o
                0x0828da44                se_ki_gasyan
 .rodata        0x0828da54       0x38 se_tk_warpin.o
                0x0828da80                se_tk_warpin
 .rodata        0x0828da8c       0x40 se_tk_warpout.o
                0x0828dac0                se_tk_warpout
 .rodata        0x0828dacc       0x2c se_tu_saa.o
                0x0828daec                se_tu_saa
 .rodata        0x0828daf8       0x3c se_hi_turun.o
                0x0828db28                se_hi_turun
 .rodata        0x0828db34       0xb0 se_track_move.o
                0x0828dbd4                se_track_move
 .rodata        0x0828dbe4       0x7c se_track_stop.o
                0x0828dc4c                se_track_stop
 .rodata        0x0828dc60       0x24 se_track_haiki.o
                0x0828dc78                se_track_haiki
 .rodata        0x0828dc84       0x38 se_track_door.o
                0x0828dcac                se_track_door
 .rodata        0x0828dcbc       0x28 se_moter.o
                0x0828dcd8                se_moter
 .rodata        0x0828dce4       0x60 se_card.o
                0x0828dd38                se_card
 .rodata        0x0828dd44       0x48 se_save.o
                0x0828dd7c                se_save
 .rodata        0x0828dd8c       0x2c se_kon.o
                0x0828dda8                se_kon
 .rodata        0x0828ddb8       0x2c se_kon2.o
                0x0828ddd4                se_kon2
 .rodata        0x0828dde4       0x2c se_kon3.o
                0x0828de00                se_kon3
 .rodata        0x0828de10       0x2c se_kon4.o
                0x0828de2c                se_kon4
 .rodata        0x0828de3c       0x54 se_suikomu.o
                0x0828de80                se_suikomu
 .rodata        0x0828de90       0x40 se_nageru.o
                0x0828dec4                se_nageru
 .rodata        0x0828ded0       0x38 se_toy_c.o
                0x0828def8                se_toy_c
 .rodata        0x0828df08       0x38 se_toy_d.o
                0x0828df30                se_toy_d
 .rodata        0x0828df40       0x38 se_toy_e.o
                0x0828df68                se_toy_e
 .rodata        0x0828df78       0x38 se_toy_f.o
                0x0828dfa0                se_toy_f
 .rodata        0x0828dfb0       0x38 se_toy_g.o
                0x0828dfd8                se_toy_g
 .rodata        0x0828dfe8       0x38 se_toy_a.o
                0x0828e010                se_toy_a
 .rodata        0x0828e020       0x38 se_toy_b.o
                0x0828e048                se_toy_b
 .rodata        0x0828e058       0x38 se_toy_c1.o
                0x0828e080                se_toy_c1
 .rodata        0x0828e090       0x30 se_mizu.o
                0x0828e0b4                se_mizu
 .rodata        0x0828e0c0       0x24 se_hashi.o
                0x0828e0d8                se_hashi
 .rodata        0x0828e0e4       0x50 se_daugi.o
                0x0828e124                se_daugi
 .rodata        0x0828e134       0x60 se_pinpon.o
                0x0828e184                se_pinpon
 .rodata        0x0828e194       0x30 se_fuusen1.o
                0x0828e1b8                se_fuusen1
 .rodata        0x0828e1c4       0x30 se_fuusen2.o
                0x0828e1e8                se_fuusen2
 .rodata        0x0828e1f4       0x38 se_fuusen3.o
                0x0828e220                se_fuusen3
 .rodata        0x0828e22c       0x44 se_toy_kabe.o
                0x0828e264                se_toy_kabe
 .rodata        0x0828e270       0x30 se_toy_dango.o
                0x0828e294                se_toy_dango
 .rodata        0x0828e2a0       0x28 se_doku.o
                0x0828e2bc                se_doku
 .rodata        0x0828e2c8       0x68 se_esuka.o
                0x0828e324                se_esuka
 .rodata        0x0828e330       0x3c se_t_ame.o
                0x0828e360                se_t_ame
 .rodata        0x0828e36c       0x40 se_t_ame_e.o
                0x0828e3a0                se_t_ame_e
 .rodata        0x0828e3ac       0x3c se_t_ooame.o
                0x0828e3dc                se_t_ooame
 .rodata        0x0828e3e8       0x40 se_t_ooame_e.o
                0x0828e41c                se_t_ooame_e
 .rodata        0x0828e428       0x3c se_t_koame.o
                0x0828e458                se_t_koame
 .rodata        0x0828e464       0x40 se_t_koame_e.o
                0x0828e498                se_t_koame_e
 .rodata        0x0828e4a4       0x68 se_t_kami.o
                0x0828e500                se_t_kami
 .rodata        0x0828e50c       0x50 se_t_kami2.o
                0x0828e550                se_t_kami2
 .rodata        0x0828e55c       0x40 se_elebeta.o
                0x0828e58c                se_elebeta
 .rodata        0x0828e59c       0x2c se_hinsi.o
                0x0828e5bc                se_hinsi
 .rodata        0x0828e5c8       0x50 se_expmax.o
                0x0828e608                se_expmax
 .rodata        0x0828e618       0x20 se_tamakoro.o
                0x0828e62c                se_tamakoro
 .rodata        0x0828e638       0x54 se_tamakoro_e.o
                0x0828e680                se_tamakoro_e
 .rodata        0x0828e68c       0x98 se_basabasa.o
                0x0828e714                se_basabasa
 .rodata        0x0828e724       0x3c se_regi.o
                0x0828e750                se_regi
 .rodata        0x0828e760       0x20 se_c_gaji.o
                0x0828e774                se_c_gaji
 .rodata        0x0828e780       0x68 se_c_maku_u.o
                0x0828e7d8                se_c_maku_u
 .rodata        0x0828e7e8       0x68 se_c_maku_d.o
                0x0828e840                se_c_maku_d
 .rodata        0x0828e850       0x24 se_c_pasi.o
                0x0828e868                se_c_pasi
 .rodata        0x0828e874       0x34 se_c_syu.o
                0x0828e89c                se_c_syu
 .rodata        0x0828e8a8       0x2c se_c_pikon.o
                0x0828e8c8                se_c_pikon
 .rodata        0x0828e8d4       0x7c se_reapoke.o
                0x0828e944                se_reapoke
 .rodata        0x0828e950       0xc0 se_op_basyu.o
                0x0828ea04                se_op_basyu
 .rodata        0x0828ea10       0xec se_bt_start.o
                0x0828eaec                se_bt_start
 .rodata        0x0828eafc      0x114 se_dendou.o
                0x0828ec04                se_dendou
 .rodata        0x0828ec10       0x24 se_jihanki.o
                0x0828ec28                se_jihanki
 .rodata        0x0828ec34      0x118 se_tama.o
                0x0828ed3c                se_tama
 .rodata        0x0828ed4c       0x28 se_z_scroll.o
                0x0828ed68                se_z_scroll
 .rodata        0x0828ed74       0x34 se_z_page.o
                0x0828ed9c                se_z_page
 .rodata        0x0828eda8       0x68 se_pn_on.o
                0x0828ee00                se_pn_on
 .rodata        0x0828ee10       0x68 se_pn_off.o
                0x0828ee68                se_pn_off
 .rodata        0x0828ee78      0x1fc se_z_search.o
                0x0828f064                se_z_search
 .rodata        0x0828f074       0x8c se_tamago.o
                0x0828f0f0                se_tamago
 .rodata        0x0828f100       0x50 se_tb_start.o
                0x0828f140                se_tb_start
 .rodata        0x0828f150       0x28 se_tb_kon.o
                0x0828f16c                se_tb_kon
 .rodata        0x0828f178       0x20 se_tb_kara.o
                0x0828f18c                se_tb_kara
 .rodata        0x0828f198       0x3c se_bidoro.o
                0x0828f1c8                se_bidoro
 .rodata        0x0828f1d4       0x98 se_w085.o
                0x0828f25c                se_w085
 .rodata        0x0828f26c       0x6c se_w085b.o
                0x0828f2c8                se_w085b
 .rodata        0x0828f2d8       0x48 se_w231.o
                0x0828f310                se_w231
 .rodata        0x0828f320       0xc4 se_w171.o
                0x0828f3d4                se_w171
 .rodata        0x0828f3e4       0x54 se_w233.o
                0x0828f428                se_w233
 .rodata        0x0828f438       0x80 se_w233b.o
                0x0828f4a8                se_w233b
 .rodata        0x0828f4b8       0x34 se_w145.o
                0x0828f4e0                se_w145
 .rodata        0x0828f4ec       0x38 se_w145b.o
                0x0828f514                se_w145b
 .rodata        0x0828f524       0x3c se_w145c.o
                0x0828f554                se_w145c
 .rodata        0x0828f560       0x78 se_w240.o
                0x0828f5cc                se_w240
 .rodata        0x0828f5d8       0x84 se_w015.o
                0x0828f64c                se_w015
 .rodata        0x0828f65c       0x54 se_w081.o
                0x0828f6a4                se_w081
 .rodata        0x0828f6b0       0xa8 se_w081b.o
                0x0828f748                se_w081b
 .rodata        0x0828f758       0x48 se_w088.o
                0x0828f794                se_w088
 .rodata        0x0828f7a0       0x7c se_w016.o
                0x0828f810                se_w016
 .rodata        0x0828f81c       0x4c se_w016b.o
                0x0828f85c                se_w016b
 .rodata        0x0828f868       0x34 se_w003.o
                0x0828f890                se_w003
 .rodata        0x0828f89c       0x4c se_w104.o
                0x0828f8dc                se_w104
 .rodata        0x0828f8e8       0x64 se_w013.o
                0x0828f93c                se_w013
 .rodata        0x0828f94c       0x4c se_w196.o
                0x0828f988                se_w196
 .rodata        0x0828f998       0x84 se_w086.o
                0x0828fa0c                se_w086
 .rodata        0x0828fa1c       0x54 se_w004.o
                0x0828fa60                se_w004
 .rodata        0x0828fa70       0xc8 se_w025.o
                0x0828fb2c                se_w025
 .rodata        0x0828fb38       0xa4 se_w025b.o
                0x0828fbcc                se_w025b
 .rodata        0x0828fbdc       0x38 se_w152.o
                0x0828fc08                se_w152
 .rodata        0x0828fc14       0x4c se_w026.o
                0x0828fc54                se_w026
 .rodata        0x0828fc60       0x88 se_w172.o
                0x0828fcd8                se_w172
 .rodata        0x0828fce8       0x70 se_w172b.o
                0x0828fd48                se_w172b
 .rodata        0x0828fd58       0xd4 se_w053.o
                0x0828fe1c                se_w053
 .rodata        0x0828fe2c       0xa4 se_w007.o
                0x0828fec0                se_w007
 .rodata        0x0828fed0       0x6c se_w092.o
                0x0828ff30                se_w092
 .rodata        0x0828ff3c       0x78 se_w221.o
                0x0828ffa4                se_w221
 .rodata        0x0828ffb4       0xe0 se_w221b.o
                0x08290084                se_w221b
 .rodata        0x08290094       0x38 se_w052.o
                0x082900c0                se_w052
 .rodata        0x082900cc       0x68 se_w036.o
                0x08290128                se_w036
 .rodata        0x08290134       0x7c se_w059.o
                0x082901a4                se_w059
 .rodata        0x082901b0       0x4c se_w059b.o
                0x082901f0                se_w059b
 .rodata        0x082901fc       0x48 se_w010.o
                0x08290238                se_w010
 .rodata        0x08290244       0x6c se_w011.o
                0x082902a0                se_w011
 .rodata        0x082902b0       0x9c se_w017.o
                0x0829033c                se_w017
 .rodata        0x0829034c      0x164 se_w019.o
                0x082904a0                se_w019
 .rodata        0x082904b0       0x68 se_w028.o
                0x08290508                se_w028
 .rodata        0x08290518       0x40 se_w013b.o
                0x0829054c                se_w013b
 .rodata        0x08290558       0x80 se_w044.o
                0x082905c8                se_w044
 .rodata        0x082905d8       0x68 se_w029.o
                0x08290634                se_w029
 .rodata        0x08290640       0x80 se_w057.o
                0x082906b4                se_w057
 .rodata        0x082906c0       0x84 se_w056.o
                0x08290734                se_w056
 .rodata        0x08290744       0x98 se_w250.o
                0x082907d0                se_w250
 .rodata        0x082907dc       0x4c se_w030.o
                0x0829081c                se_w030
 .rodata        0x08290828       0x40 se_w039.o
                0x0829085c                se_w039
 .rodata        0x08290868       0x78 se_w054.o
                0x082908d4                se_w054
 .rodata        0x082908e0       0x3c se_w077.o
                0x08290910                se_w077
 .rodata        0x0829091c       0x58 se_w020.o
                0x08290968                se_w020
 .rodata        0x08290974       0xc8 se_w082.o
                0x08290a30                se_w082
 .rodata        0x08290a3c       0xf8 se_w047.o
                0x08290b24                se_w047
 .rodata        0x08290b34      0x110 se_w195.o
                0x08290c34                se_w195
 .rodata        0x08290c44       0x84 se_w006.o
                0x08290cbc                se_w006
 .rodata        0x08290cc8       0x48 se_w091.o
                0x08290d04                se_w091
 .rodata        0x08290d10       0x60 se_w146.o
                0x08290d64                se_w146
 .rodata        0x08290d70       0x4c se_w120.o
                0x08290db0                se_w120
 .rodata        0x08290dbc       0x8c se_w153.o
                0x08290e38                se_w153
 .rodata        0x08290e48       0xbc se_w071b.o
                0x08290ef4                se_w071b
 .rodata        0x08290f04       0x54 se_w071.o
                0x08290f4c                se_w071
 .rodata        0x08290f58       0x80 se_w103.o
                0x08290fc8                se_w103
 .rodata        0x08290fd8       0xc4 se_w062.o
                0x08291090                se_w062
 .rodata        0x0829109c       0xbc se_w062b.o
                0x0829114c                se_w062b
 .rodata        0x08291158       0xec se_w048.o
                0x08291238                se_w048
 .rodata        0x08291244       0x40 se_w187.o
                0x08291278                se_w187
 .rodata        0x08291284       0x5c se_w118.o
                0x082912d4                se_w118
 .rodata        0x082912e0       0x38 se_w155.o
                0x0829130c                se_w155
 .rodata        0x08291318       0xb4 se_w122.o
                0x082913c0                se_w122
 .rodata        0x082913cc       0xa4 se_w060.o
                0x08291460                se_w060
 .rodata        0x08291470       0x64 se_w185.o
                0x082914c8                se_w185
 .rodata        0x082914d4      0x128 se_w014.o
                0x082915ec                se_w014
 .rodata        0x082915fc       0x7c se_w043.o
                0x08291668                se_w043
 .rodata        0x08291678       0x58 se_w207.o
                0x082916c4                se_w207
 .rodata        0x082916d0       0x38 se_w207b.o
                0x082916fc                se_w207b
 .rodata        0x08291708       0x50 se_w215.o
                0x0829174c                se_w215
 .rodata        0x08291758       0x8c se_w109.o
                0x082917d8                se_w109
 .rodata        0x082917e4       0x68 se_w173.o
                0x0829183c                se_w173
 .rodata        0x0829184c       0x78 se_w280.o
                0x082918b4                se_w280
 .rodata        0x082918c4       0x64 se_w202.o
                0x0829191c                se_w202
 .rodata        0x08291928      0x154 se_w060b.o
                0x08291a70                se_w060b
 .rodata        0x08291a7c       0xd4 se_w076.o
                0x08291b44                se_w076
 .rodata        0x08291b50      0x114 se_w080.o
                0x08291c54                se_w080
 .rodata        0x08291c64       0xe0 se_w100.o
                0x08291d38                se_w100
 .rodata        0x08291d44       0xe0 se_w107.o
                0x08291e18                se_w107
 .rodata        0x08291e24       0x4c se_w166.o
                0x08291e64                se_w166
 .rodata        0x08291e70       0x90 se_w129.o
                0x08291ef0                se_w129
 .rodata        0x08291f00      0x190 se_w115.o
                0x08292080                se_w115
 .rodata        0x08292090      0x1a0 se_w112.o
                0x08292220                se_w112
 .rodata        0x08292230       0x6c se_w197.o
                0x08292290                se_w197
 .rodata        0x0829229c       0x50 se_w199.o
                0x082922e0                se_w199
 .rodata        0x082922ec      0x128 se_w236.o
                0x08292404                se_w236
 .rodata        0x08292414       0x7c se_w204.o
                0x08292484                se_w204
 .rodata        0x08292490       0xf0 se_w268.o
                0x08292574                se_w268
 .rodata        0x08292580       0x68 se_w070.o
                0x082925d8                se_w070
 .rodata        0x082925e8       0x5c se_w063.o
                0x08292634                se_w063
 .rodata        0x08292644       0xb4 se_w127.o
                0x082926e8                se_w127
 .rodata        0x082926f8      0x1fc se_w179.o
                0x082928e4                se_w179
 .rodata        0x082928f4      0x11c se_w151.o
                0x08292a04                se_w151
 .rodata        0x08292a10      0x174 se_w201.o
                0x08292b74                se_w201
 .rodata        0x08292b84       0x70 se_w161.o
                0x08292be4                se_w161
 .rodata        0x08292bf4       0x98 se_w161b.o
                0x08292c7c                se_w161b
 .rodata        0x08292c8c       0x34 se_w227.o
                0x08292cb4                se_w227
 .rodata        0x08292cc0       0xd8 se_w227b.o
                0x08292d8c                se_w227b
 .rodata        0x08292d98       0xdc se_w226.o
                0x08292e64                se_w226
 .rodata        0x08292e74       0xac se_w208.o
                0x08292f10                se_w208
 .rodata        0x08292f20       0x98 se_w213.o
                0x08292fa8                se_w213
 .rodata        0x08292fb8       0x98 se_w213b.o
                0x08293040                se_w213b
 .rodata        0x08293050       0xa8 se_w234.o
                0x082930e8                se_w234
 .rodata        0x082930f8       0x48 se_w260.o
                0x08293134                se_w260
 .rodata        0x08293140      0x100 se_w328.o
                0x08293230                se_w328
 .rodata        0x08293240       0x94 se_w320.o
                0x082932c4                se_w320
 .rodata        0x082932d4       0x64 se_w255.o
                0x08293328                se_w255
 .rodata        0x08293338       0x9c se_w291.o
                0x082933c4                se_w291
 .rodata        0x082933d4      0x208 se_w089.o
                0x082935cc                se_w089
 .rodata        0x082935dc       0xfc se_w239.o
                0x082936c8                se_w239
 .rodata        0x082936d8       0xf0 se_w230.o
                0x082937b8                se_w230
 .rodata        0x082937c8       0x84 se_w281.o
                0x0829383c                se_w281
 .rodata        0x0829384c       0x74 se_w327.o
                0x082938b0                se_w327
 .rodata        0x082938c0      0x180 se_w287.o
                0x08293a30                se_w287
 .rodata        0x08293a40      0x104 se_w257.o
                0x08293b34                se_w257
 .rodata        0x08293b44       0x5c se_w253.o
                0x08293b94                se_w253
 .rodata        0x08293ba0       0x74 se_w258.o
                0x08293c04                se_w258
 .rodata        0x08293c14      0x11c se_w322.o
                0x08293d20                se_w322
 .rodata        0x08293d30       0xa4 se_w298.o
                0x08293dc4                se_w298
 .rodata        0x08293dd4      0x170 se_w287b.o
                0x08293f34                se_w287b
 .rodata        0x08293f44      0x134 se_w114.o
                0x08294068                se_w114
 .rodata        0x08294078       0x84 se_w063b.o
                0x082940ec                se_w063b
 .rodata        0x082940fc       0x58 se_rg_w_door.o
                0x08294144                se_rg_w_door
 .rodata        0x08294154       0x2c se_rg_card1.o
                0x08294174                se_rg_card1
 .rodata        0x08294180       0x38 se_rg_card2.o
                0x082941ac                se_rg_card2
 .rodata        0x082941b8       0x90 se_rg_card3.o
                0x08294238                se_rg_card3
 .rodata        0x08294248       0x38 se_rg_bag1.o
                0x08294270                se_rg_bag1
 .rodata        0x08294280       0x44 se_rg_bag2.o
                0x082942b4                se_rg_bag2
 .rodata        0x082942c4       0x40 se_rg_getting.o
                0x082942f4                se_rg_getting
 .rodata        0x08294304       0x24 se_rg_shop.o
                0x0829431c                se_rg_shop
 .rodata        0x08294328       0xbc se_rg_kiteki.o
                0x082943d4                se_rg_kiteki
 .rodata        0x082943e4       0x70 se_rg_help_op.o
                0x08294448                se_rg_help_op
 .rodata        0x08294454       0x6c se_rg_help_cl.o
                0x082944b4                se_rg_help_cl
 .rodata        0x082944c0       0x48 se_rg_help_ng.o
                0x082944fc                se_rg_help_ng
 .rodata        0x08294508       0xe8 se_rg_deomov.o
                0x082945dc                se_rg_deomov
 .rodata        0x082945f0       0xbc se_rg_excellent.o
                0x0829469c                se_rg_excellent
 .rodata        0x082946ac       0x30 se_rg_nawamiss.o
                0x082946d0                se_rg_nawamiss
 .rodata        0x082946dc       0xa4 se_toreeye.o
                0x08294770                se_toreeye
 .rodata        0x08294780       0x60 se_toreoff.o
                0x082947d0                se_toreoff
 .rodata        0x082947e0       0x34 se_hantei1.o
                0x08294804                se_hantei1
 .rodata        0x08294814       0x44 se_hantei2.o
                0x08294848                se_hantei2
 .rodata        0x08294858       0xd8 se_curtain.o
                0x0829491c                se_curtain
 .rodata        0x08294930       0xdc se_curtain1.o
                0x082949f8                se_curtain1
 .rodata        0x08294a0c       0x38 se_ussoki.o
                0x08294a38                se_ussoki
 .rodata        0x08294a44      0xa18 tetsuji.o
                0x08295430                tetsuji
 .rodata        0x0829545c      0x3c4 field13.o
                0x08295808                field13
 .rodata        0x08295820      0x440 kachi22.o
                0x08295c3c                kachi22
 .rodata        0x08295c60      0x530 kachi2.o
                0x0829616c                kachi2
 .rodata        0x08296190      0xef4 kachi3.o
                0x0829705c                kachi3
 .rodata        0x08297084      0xb94 kachi5.o
                0x08297bf0                kachi5
 .rodata        0x08297c18      0x2d0 pcc.o
                0x08297ed4                pcc
 .rodata        0x08297ee8      0x5c4 nibi.o
                0x08298494                nibi
 .rodata        0x082984ac      0x9d4 suikun.o
                0x08298e6c                suikun
 .rodata        0x08298e80      0x8e0 dooro1.o
                0x08299738                dooro1
 .rodata        0x08299760      0xb7c dooro_x1.o
                0x0829a2b0                dooro_x1
 .rodata        0x0829a2dc     0x1298 dooro_x3.o
                0x0829b54c                dooro_x3
 .rodata        0x0829b574      0xac4 machi_s2.o
                0x0829c010                machi_s2
 .rodata        0x0829c038      0x8e8 machi_s4.o
                0x0829c8fc                machi_s4
 .rodata        0x0829c920      0xa00 gim.o
                0x0829d2fc                gim
 .rodata        0x0829d320      0xea0 naminori.o
                0x0829e1a0                naminori
 .rodata        0x0829e1c0      0x92c dan01.o
                0x0829eac0                dan01
 .rodata        0x0829eaec       0xe4 fanfa1.o
                0x0829ebb4                fanfa1
 .rodata        0x0829ebd0       0xc8 me_asa.o
                0x0829ec80                me_asa
 .rodata        0x0829ec98      0x2d8 me_bachi.o
                0x0829ef4c                me_bachi
 .rodata        0x0829ef70      0x150 fanfa4.o
                0x0829f0a0                fanfa4
 .rodata        0x0829f0c0      0x1a0 fanfa5.o
                0x0829f23c                fanfa5
 .rodata        0x0829f260      0x18c me_waza.o
                0x0829f3c8                me_waza
 .rodata        0x0829f3ec      0xac0 bijyutu.o
                0x0829fe8c                bijyutu
 .rodata        0x0829feac      0xeb0 dooro_x4.o
                0x082a0d34                dooro_x4
 .rodata        0x082a0d5c      0xe58 fune_kan.o
                0x082a1b90                fune_kan
 .rodata        0x082a1bb4       0x68 me_shinka.o
                0x082a1c04                me_shinka
 .rodata        0x082a1c1c      0x57c shinka.o
                0x082a2174                shinka
 .rodata        0x082a2198       0xe0 me_wasure.o
                0x082a2258                me_wasure
 .rodata        0x082a2278      0x590 syoujoeye.o
                0x082a27e0                syoujoeye
 .rodata        0x082a2808      0x658 boyeye.o
                0x082a2e3c                boyeye
 .rodata        0x082a2e60      0x940 dan02.o
                0x082a3778                dan02
 .rodata        0x082a37a0      0x934 machi_s3.o
                0x082a40ac                machi_s3
 .rodata        0x082a40d4      0x6ac odamaki.o
                0x082a475c                odamaki
 .rodata        0x082a4780      0xb90 b_tower.o
                0x082a52e4                b_tower
 .rodata        0x082a5310      0x4dc swimeye.o
                0x082a57c4                swimeye
 .rodata        0x082a57ec      0x928 dan03.o
                0x082a60e8                dan03
 .rodata        0x082a6114       0xd0 me_kinomi.o
                0x082a61c8                me_kinomi
 .rodata        0x082a61e4      0x36c me_tama.o
                0x082a652c                me_tama
 .rodata        0x082a6550      0x22c me_b_big.o
                0x082a6758                me_b_big
 .rodata        0x082a677c      0x140 me_b_small.o
                0x082a6898                me_b_small
 .rodata        0x082a68bc       0xf4 me_zannen.o
                0x082a6994                me_zannen
 .rodata        0x082a69b0      0x61c bd_time.o
                0x082a6fa8                bd_time
 .rodata        0x082a6fcc      0x888 test1.o
                0x082a7830                test1
 .rodata        0x082a7854      0x944 test2.o
                0x082a8174                test2
 .rodata        0x082a8198      0x97c test3.o
                0x082a8af0                test3
 .rodata        0x082a8b14      0x89c test4.o
                0x082a9394                test4
 .rodata        0x082a93b0      0x644 test.o
                0x082a99d8                test
 .rodata        0x082a99f4      0xac4 gomachi0.o
                0x082aa488                gomachi0
 .rodata        0x082aa4b8     0x12f4 gotown.o
                0x082ab784                gotown
 .rodata        0x082ab7ac      0xc44 pokecen.o
                0x082ac3c4                pokecen
 .rodata        0x082ac3f0     0x13cc nextroad.o
                0x082ad78c                nextroad
 .rodata        0x082ad7bc     0x1d04 granroad.o
                0x082af494                granroad
 .rodata        0x082af4c0     0x17e4 cycling.o
                0x082b0c78                cycling
 .rodata        0x082b0ca4     0x12bc friendly.o
                0x082b1f38                friendly
 .rodata        0x082b1f60     0x1258 mishiro.o
                0x082b318c                mishiro
 .rodata        0x082b31b8     0x24c0 tozan.o
                0x082b564c                tozan
 .rodata        0x082b5678      0x670 girleye.o
                0x082b5cbc                girleye
 .rodata        0x082b5ce8     0x11e8 minamo.o
                0x082b6eb0                minamo
 .rodata        0x082b6ed0      0xf84 ashroad.o
                0x082b7e2c                ashroad
 .rodata        0x082b7e54      0x3d0 event0.o
                0x082b8200                event0
 .rodata        0x082b8224     0x1610 deepdeep.o
                0x082b9804                deepdeep
 .rodata        0x082b9834     0x1188 kachi1.o
                0x082ba990                kachi1
 .rodata        0x082ba9bc     0x2e08 title3.o
                0x082bd794                title3
 .rodata        0x082bd7c4     0x119c demo1.o
                0x082be930                demo1
 .rodata        0x082be960      0xd04 girl_sup.o
                0x082bf634                girl_sup
 .rodata        0x082bf664      0x92c hageshii.o
                0x082bff68                hageshii
 .rodata        0x082bff90      0xcd4 kakkoii.o
                0x082c0c38                kakkoii
 .rodata        0x082c0c64     0x1744 kazanbai.o
                0x082c237c                kazanbai
 .rodata        0x082c23a8      0xe40 aqa_0.o
                0x082c31b8                aqa_0
 .rodata        0x082c31e8      0x630 tsuretek.o
                0x082c37f0                tsuretek
 .rodata        0x082c3818      0xd04 boy_sup.o
                0x082c44ec                boy_sup
 .rodata        0x082c451c      0xe00 rainbow.o
                0x082c52f4                rainbow
 .rodata        0x082c531c      0x8cc ayasii.o
                0x082c5bbc                ayasii
 .rodata        0x082c5be8      0x4d0 kachi4.o
                0x082c608c                kachi4
 .rodata        0x082c60b8      0x674 ropeway.o
                0x082c6700                ropeway
 .rodata        0x082c672c     0x1728 casino.o
                0x082c7e24                casino
 .rodata        0x082c7e54      0xe4c hightown.o
                0x082c8c70                hightown
 .rodata        0x082c8ca0      0x78c safari.o
                0x082c9400                safari
 .rodata        0x082c942c     0x13a0 c_road.o
                0x082ca79c                c_road
 .rodata        0x082ca7cc      0x90c ajito.o
                0x082cb0ac                ajito
 .rodata        0x082cb0d8      0xe08 m_boat.o
                0x082cbeb4                m_boat
 .rodata        0x082cbee0      0xcb4 m_dungon.o
                0x082ccb64                m_dungon
 .rodata        0x082ccb94     0x1e3c finecity.o
                0x082ce9a0                finecity
 .rodata        0x082ce9d0     0x2254 machupi.o
                0x082d0bf4                machupi
 .rodata        0x082d0c24      0x348 p_school.o
                0x082d0f54                p_school
 .rodata        0x082d0f6c      0xbb0 dendou.o
                0x082d1aec                dendou
 .rodata        0x082d1b1c      0xeb8 tonekusa.o
                0x082d29a8                tonekusa
 .rodata        0x082d29d4      0x810 maborosi.o
                0x082d31bc                maborosi
 .rodata        0x082d31e4      0x60c con_fan.o
                0x082d37c8                con_fan
 .rodata        0x082d37f0      0xec4 contest0.o
                0x082d468c                contest0
 .rodata        0x082d46b4      0xb68 mgm0.o
                0x082d51ec                mgm0
 .rodata        0x082d521c      0xc20 t_battle.o
                0x082d5e10                t_battle
 .rodata        0x082d5e3c      0x654 ooame.o
                0x082d6470                ooame
 .rodata        0x082d6490      0x2d0 hideri.o
                0x082d674c                hideri
 .rodata        0x082d6760     0x10f0 runecity.o
                0x082d7828                runecity
 .rodata        0x082d7850      0x464 con_k.o
                0x082d7c8c                con_k
 .rodata        0x082d7cb4      0x7b8 eikou_r.o
                0x082d8448                eikou_r
 .rodata        0x082d846c      0xee4 karakuri.o
                0x082d9328                karakuri
 .rodata        0x082d9350      0x510 hutago.o
                0x082d9830                hutago
 .rodata        0x082d9860      0xc84 sitennou.o
                0x082da4b8                sitennou
 .rodata        0x082da4e4      0x580 yama_eye.o
                0x082daa3c                yama_eye
 .rodata        0x082daa64      0x688 conlobby.o
                0x082db0c4                conlobby
 .rodata        0x082db0ec      0x588 inter_v.o
                0x082db648                inter_v
 .rodata        0x082db674     0x10ec daigo.o
                0x082dc730                daigo
 .rodata        0x082dc760     0x262c thankfor.o
                0x082ded5c                thankfor
 .rodata        0x082ded8c      0x504 end.o
                0x082df280                end
 .rodata        0x082df290     0x13c0 mus_b_frontier.o
                0x082e0624                mus_b_frontier
 .rodata        0x082e0650      0xc90 mus_b_arena.o
                0x082e12b4                mus_b_arena
 .rodata        0x082e12e0      0x308 me_pointget.o
                0x082e15bc                me_pointget
 .rodata        0x082e15e8      0x114 me_tore_eye.o
                0x082e16e0                me_tore_eye
 .rodata        0x082e16fc     0x22b0 mus_pyramid.o
                0x082e397c                mus_pyramid
 .rodata        0x082e39ac      0x3ec mus_pyramid_top.o
                0x082e3d74                mus_pyramid_top
 .rodata        0x082e3d98     0x1590 mus_b_palace.o
                0x082e52fc                mus_b_palace
 .rodata        0x082e5328      0x460 mus_rekkuu_kourin.o
                0x082e5764                mus_rekkuu_kourin
 .rodata        0x082e5788     0x1334 mus_sattower.o
                0x082e6a98                mus_sattower
 .rodata        0x082e6abc      0x3cc me_symbolget.o
                0x082e6e5c                me_symbolget
 .rodata        0x082e6e88     0x14fc mus_b_dome.o
                0x082e8354                mus_b_dome
 .rodata        0x082e8384     0x147c mus_b_tube.o
                0x082e97d0                mus_b_tube
 .rodata        0x082e9800     0x1eac mus_b_factory.o
                0x082eb680                mus_b_factory
 .rodata        0x082eb6ac      0x6e8 mus_vs_rekku.o
                0x082ebd74                mus_vs_rekku
 .rodata        0x082ebd94     0x275c mus_vs_front.o
                0x082ee4c0                mus_vs_front
 .rodata        0x082ee4f0     0x14b4 mus_vs_mew.o
                0x082ef97c                mus_vs_mew
 .rodata        0x082ef9a4      0x24c mus_b_dome1.o
                0x082efbdc                mus_b_dome1
 .rodata        0x082efbf0      0xad0 battle27.o
                0x082f0698                battle27
 .rodata        0x082f06c0     0x1268 battle31.o
                0x082f1900                battle31
 .rodata        0x082f1928     0x10a4 battle20.o
                0x082f29a4                battle20
 .rodata        0x082f29cc      0xe30 battle32.o
                0x082f37d4                battle32
 .rodata        0x082f37fc      0xef0 battle33.o
                0x082f46c4                battle33
 .rodata        0x082f46ec      0x914 battle36.o
                0x082f4fd8                battle36
 .rodata        0x082f5000      0x6e8 battle34.o
                0x082f56c8                battle34
 .rodata        0x082f56e8      0xcb0 battle35.o
                0x082f6370                battle35
 .rodata        0x082f6398      0xc30 battle38.o
                0x082f6fa0                battle38
 .rodata        0x082f6fc8      0xe98 battle30.o
                0x082f7e38                battle30
 .rodata        0x082f7e60      0x4f4 mus_rg_annai.o
                0x082f832c                mus_rg_annai
 .rodata        0x082f8354      0xf3c mus_rg_slot.o
                0x082f9268                mus_rg_slot
 .rodata        0x082f9290     0x1c2c mus_rg_ajito.o
                0x082fae8c                mus_rg_ajito
 .rodata        0x082faebc      0xa00 mus_rg_gym.o
                0x082fb898                mus_rg_gym
 .rodata        0x082fb8bc      0x28c mus_rg_purin.o
                0x082fbb30                mus_rg_purin
 .rodata        0x082fbb48      0xb10 mus_rg_demo.o
                0x082fc630                mus_rg_demo
 .rodata        0x082fc658     0x107c mus_rg_title.o
                0x082fd6a4                mus_rg_title
 .rodata        0x082fd6d4      0xed0 mus_rg_guren.o
                0x082fe578                mus_rg_guren
 .rodata        0x082fe5a4      0xd28 mus_rg_shion.o
                0x082ff2a4                mus_rg_shion
 .rodata        0x082ff2cc       0x3c mus_rg_kaihuku.o
                0x082ff2f8                mus_rg_kaihuku
 .rodata        0x082ff308      0xc2c mus_rg_cycling.o
                0x082fff0c                mus_rg_cycling
 .rodata        0x082fff34      0x3bc mus_rg_rocket.o
                0x083002cc                mus_rg_rocket
 .rodata        0x083002f0      0x3c0 mus_rg_shoujo.o
                0x08300684                mus_rg_shoujo
 .rodata        0x083006b0      0x4a4 mus_rg_shounen.o
                0x08300b2c                mus_rg_shounen
 .rodata        0x08300b54      0xac0 mus_rg_dendou.o
                0x083015e8                mus_rg_dendou
 .rodata        0x08301614     0x121c mus_rg_t_mori.o
                0x08302800                mus_rg_t_mori
 .rodata        0x08302830     0x1444 mus_rg_otsukimi.o
                0x08303c50                mus_rg_otsukimi
 .rodata        0x08303c74     0x1248 mus_rg_pokeyashi.o
                0x08304e8c                mus_rg_pokeyashi
 .rodata        0x08304ebc     0x400c mus_rg_ending.o
                0x08308e9c                mus_rg_ending
 .rodata        0x08308ec8      0xa84 mus_rg_load01.o
                0x08309924                mus_rg_load01
 .rodata        0x0830994c      0x868 mus_rg_opening.o
                0x0830a194                mus_rg_opening
 .rodata        0x0830a1b4      0xf48 mus_rg_load02.o
                0x0830b0d0                mus_rg_load02
 .rodata        0x0830b0fc      0xd78 mus_rg_load03.o
                0x0830be44                mus_rg_load03
 .rodata        0x0830be74      0xd38 mus_rg_champ_r.o
                0x0830cb84                mus_rg_champ_r
 .rodata        0x0830cbac     0x1aec mus_rg_vs_gym.o
                0x0830e668                mus_rg_vs_gym
 .rodata        0x0830e698     0x2b74 mus_rg_vs_tore.o
                0x083111dc                mus_rg_vs_tore
 .rodata        0x0831120c     0x1174 mus_rg_vs_yasei.o
                0x08312358                mus_rg_vs_yasei
 .rodata        0x08312380     0x27d8 mus_rg_vs_last.o
                0x08314b28                mus_rg_vs_last
 .rodata        0x08314b58      0x854 mus_rg_masara.o
                0x0831538c                mus_rg_masara
 .rodata        0x083153ac      0x79c mus_rg_kenkyu.o
                0x08315b28                mus_rg_kenkyu
 .rodata        0x08315b48      0x998 mus_rg_ohkido.o
                0x083164b4                mus_rg_ohkido
 .rodata        0x083164e0      0xa64 mus_rg_pokecen.o
                0x08316f14                mus_rg_pokecen
 .rodata        0x08316f44     0x12a4 mus_rg_santoan.o
                0x083181b8                mus_rg_santoan
 .rodata        0x083181e8      0x96c mus_rg_naminori.o
                0x08318b30                mus_rg_naminori
 .rodata        0x08318b54      0x8c8 mus_rg_p_tower.o
                0x083193fc                mus_rg_p_tower
 .rodata        0x0831941c     0x1700 mus_rg_shiruhu.o
                0x0831aaf0                mus_rg_shiruhu
 .rodata        0x0831ab1c      0xa3c mus_rg_hanada.o
                0x0831b52c                mus_rg_hanada
 .rodata        0x0831b558      0xb78 mus_rg_tamamusi.o
                0x0831c0ac                mus_rg_tamamusi
 .rodata        0x0831c0d0     0x1188 mus_rg_win_tre.o
                0x0831d22c                mus_rg_win_tre
 .rodata        0x0831d258      0x530 mus_rg_win_yasei.o
                0x0831d764                mus_rg_win_yasei
 .rodata        0x0831d788      0xef4 mus_rg_win_gym.o
                0x0831e654                mus_rg_win_gym
 .rodata        0x0831e67c      0xe18 mus_rg_kuchiba.o
                0x0831f468                mus_rg_kuchiba
 .rodata        0x0831f494      0xef0 mus_rg_nibi.o
                0x08320358                mus_rg_nibi
 .rodata        0x08320384      0x83c mus_rg_rival1.o
                0x08320b94                mus_rg_rival1
 .rodata        0x08320bc0      0x7d4 mus_rg_rival2.o
                0x08321368                mus_rg_rival2
 .rodata        0x08321394      0x1f8 mus_rg_fan2.o
                0x08321568                mus_rg_fan2
 .rodata        0x0832158c      0x1fc mus_rg_fan5.o
                0x08321768                mus_rg_fan5
 .rodata        0x08321788      0x378 mus_rg_fan6.o
                0x08321ad8                mus_rg_fan6
 .rodata        0x08321b00      0x164 me_rg_photo.o
                0x08321c48                me_rg_photo
 .rodata        0x08321c64      0x904 mus_rg_titlerog.o
                0x0832254c                mus_rg_titlerog
 .rodata        0x08322568      0x440 mus_rg_get_yasei.o
                0x08322984                mus_rg_get_yasei
 .rodata        0x083229a8       0x74 mus_rg_sousa.o
                0x08322a10                mus_rg_sousa
 .rodata        0x08322a1c      0x1e4 mus_rg_sekaikan.o
                0x08322be0                mus_rg_sekaikan
 .rodata        0x08322c00       0xc0 mus_rg_seibetu.o
                0x08322c9c                mus_rg_seibetu
 .rodata        0x08322cc0      0xf78 mus_rg_jump.o
                0x08323c10                mus_rg_jump
 .rodata        0x08323c38      0xf7c mus_rg_union.o
                0x08324b8c                mus_rg_union
 .rodata        0x08324bb4      0xa64 mus_rg_network.o
                0x083255e8                mus_rg_network
 .rodata        0x08325618      0x474 mus_rg_okurimono.o
                0x08325a68                mus_rg_okurimono
 .rodata        0x08325a8c      0xf30 mus_rg_kinomikui.o
                0x08326994                mus_rg_kinomikui
 .rodata        0x083269bc     0x1400 mus_rg_nanadungeon.o
                0x08327d98                mus_rg_nanadungeon
 .rodata        0x08327dbc      0x4f4 mus_rg_oshie_tv.o
                0x08328288                mus_rg_oshie_tv
 .rodata        0x083282b0      0xec8 mus_rg_nanashima.o
                0x08329148                mus_rg_nanashima
 .rodata        0x08329178     0x121c mus_rg_nanaiseki.o
                0x0832a364                mus_rg_nanaiseki
 .rodata        0x0832a394      0xef0 mus_rg_nana123.o
                0x0832b258                mus_rg_nana123
 .rodata        0x0832b284     0x1028 mus_rg_nana45.o
                0x0832c280                mus_rg_nana45
 .rodata        0x0832c2ac      0xf30 mus_rg_nana67.o
                0x0832d1b0                mus_rg_nana67
 .rodata        0x0832d1dc      0x1a8 mus_rg_pokefue.o
                0x0832d374                mus_rg_pokefue
 .rodata        0x0832d384     0x21a8 mus_rg_vs_deo.o
                0x0832f4fc                mus_rg_vs_deo
 .rodata        0x0832f52c     0x1170 mus_rg_vs_myu2.o
                0x08330674                mus_rg_vs_myu2
 .rodata        0x0833069c     0x12b8 mus_rg_vs_den.o
                0x0833192c                mus_rg_vs_den
 .rodata        0x08331954      0x440 mus_rg_exeye.o
                0x08331d70                mus_rg_exeye
 .rodata        0x08331d94      0x948 mus_rg_deoeye.o
                0x083326b8                mus_rg_deoeye
 .rodata        0x083326dc      0xa00 mus_rg_t_tower.o
                0x083330b8                mus_rg_t_tower
 .rodata        0x083330dc      0x83c mus_rg_slowmasara.o
                0x083338f8                mus_rg_slowmasara
 .rodata        0x08333918       0xd4 mus_rg_tvnoize.o
                0x083339d4                mus_rg_tvnoize
 .rodata        0x083339ec       0x1c seq_01_1.o
                0x083339fc                seq_01_1
 .rodata        0x08333a08       0x24 seq_01_2.o
                0x08333a20                seq_01_2
 .rodata        0x08333a2c       0x1c seq_01_3.o
                0x08333a3c                seq_01_3
 .rodata        0x08333a48       0x1c seq_02_1.o
                0x08333a58                seq_02_1
 .rodata        0x08333a64       0x24 seq_02_2.o
                0x08333a7c                seq_02_2
 .rodata        0x08333a88       0x1c seq_02_3.o
                0x08333a98                seq_02_3
 .rodata        0x08333aa4       0x1c seq_03_1.o
                0x08333ab4                seq_03_1
 .rodata        0x08333ac0       0x24 seq_03_2.o
                0x08333ad8                seq_03_2
 .rodata        0x08333ae4       0x1c seq_03_3.o
                0x08333af4                seq_03_3
 .rodata        0x08333b00       0x1c seq_04_1.o
                0x08333b10                seq_04_1
 .rodata        0x08333b1c       0x24 seq_04_2.o
                0x08333b34                seq_04_2
 .rodata        0x08333b40       0x1c seq_04_3.o
                0x08333b50                seq_04_3
 .rodata        0x08333b5c       0x1c seq_05_1.o
                0x08333b6c                seq_05_1
 .rodata        0x08333b78       0x24 seq_05_2.o
                0x08333b90                seq_05_2
 .rodata        0x08333b9c       0x1c seq_05_3.o
                0x08333bac                seq_05_3
 .rodata        0x08333bb8       0x1c seq_06_1.o
                0x08333bc8                seq_06_1
 .rodata        0x08333bd4       0x24 seq_06_2.o
                0x08333bec                seq_06_2
 .rodata        0x08333bf8       0x1c seq_06_3.o
                0x08333c08                seq_06_3
 .rodata        0x08333c14       0x1c seq_07_1.o
                0x08333c24                seq_07_1
 .rodata        0x08333c30       0x24 seq_07_2.o
                0x08333c48                seq_07_2
 .rodata        0x08333c54       0x1c seq_07_3.o
                0x08333c64                seq_07_3
 .rodata        0x08333c70       0x1c seq_08_1.o
                0x08333c80                seq_08_1
 .rodata        0x08333c8c       0x24 seq_08_2.o
                0x08333ca4                seq_08_2
 .rodata        0x08333cb0       0x1c seq_08_3.o
                0x08333cc0                seq_08_3
 .rodata        0x08333ccc       0x1c seq_09_1.o
                0x08333cdc                seq_09_1
 .rodata        0x08333ce8       0x24 seq_09_2.o
                0x08333d00                seq_09_2
 .rodata        0x08333d0c       0x1c seq_09_3.o
                0x08333d1c                seq_09_3
 .rodata        0x08333d28       0x1c seq_10_1.o
                0x08333d38                seq_10_1
 .rodata        0x08333d44       0x24 seq_10_2.o
                0x08333d5c                seq_10_2
 .rodata        0x08333d68       0x1c seq_10_3.o
                0x08333d78                seq_10_3
 .rodata        0x08333d84       0x1c seq_11_1.o
                0x08333d94                seq_11_1
 .rodata        0x08333da0       0x24 seq_11_2.o
                0x08333db8                seq_11_2
 .rodata        0x08333dc4       0x1c seq_11_3.o
                0x08333dd4                seq_11_3
 .rodata        0x08333de0       0x1c seq_12_1.o
                0x08333df0                seq_12_1
 .rodata        0x08333dfc       0x24 seq_12_2.o
                0x08333e14                seq_12_2
 .rodata        0x08333e20       0x1c seq_12_3.o
                0x08333e30                seq_12_3
 .rodata        0x08333e3c       0x1c seq_13_1.o
                0x08333e4c                seq_13_1
 .rodata        0x08333e58       0x24 seq_13_2.o
                0x08333e70                seq_13_2
 .rodata        0x08333e7c       0x1c seq_13_3.o
                0x08333e8c                seq_13_3
 .rodata        0x08333e98       0x1c seq_14_1.o
                0x08333ea8                seq_14_1
 .rodata        0x08333eb4       0x24 seq_14_2.o
                0x08333ecc                seq_14_2
 .rodata        0x08333ed8       0x1c seq_14_3.o
                0x08333ee8                seq_14_3
 .rodata        0x08333ef4       0x1c seq_15_1.o
                0x08333f04                seq_15_1
 .rodata        0x08333f10       0x24 seq_15_2.o
                0x08333f28                seq_15_2
 .rodata        0x08333f34       0x1c seq_15_3.o
                0x08333f44                seq_15_3
 .rodata        0x08333f50       0x1c seq_16_1.o
                0x08333f60                seq_16_1
 .rodata        0x08333f6c       0x24 seq_16_2.o
                0x08333f84                seq_16_2
 .rodata        0x08333f90       0x1c seq_16_3.o
                0x08333fa0                seq_16_3
 .rodata        0x08333fac       0x1c seq_17_1.o
                0x08333fbc                seq_17_1
 .rodata        0x08333fc8       0x24 seq_17_2.o
                0x08333fe0                seq_17_2
 .rodata        0x08333fec       0x1c seq_17_3.o
                0x08333ffc                seq_17_3
 *(.rodata.*)
 .rodata.end    0x08334008        0x4 E:\pm3sound20041208\pm3sound\SndMonDat.o
                0x08334008                seg_rodata_end
 *(.gnu.linkonce.r*)

.rodata1
 *(.rodata1)
                0x0833410c                .=(ALIGN(0x100)+(.&0xff))

.data           0x0833410c        0x0
 *(.data)
 *(.data.*)
 *(.gnu.linkonce.d*)

.data1
 *(.data1)

.ctors
 EXCLUDE_FILE ( *crtend.o )*(.ctors)
 *(SORT(.ctors.*))
 *crtend(.ctors)

.dtors
 EXCLUDE_FILE ( *crtend.o )*(.dtors)
 *(SORT(.dtors.*))
 *crtend.o(.dtors)

.got
 *(.got.plt)
 *(.got)

.dynamic
 *(.dynamic)

.sdata
 *(.sdata)
 *(.sdata.*)
                0x0833410c                _edata=.
                0x0833410c                PROVIDE (edata, .)
                0x0833410c                __bss_start=.
                0x0833410c                __bss_start__=.

.sbss
 *(.sbss)
 *(.scommon)

.bss            0x03000000     0x3f30
 *(.dynbss)
 *(.bss)
 .bss           0x03000000       0x40 m4aLib.o
 .bss           0x03000040      0x730 SoundDat.o
 *(.bss.*)
 .bss.code      0x03000770      0x800 m4aLib.o
                0x03000770                SoundMainBuf
 *(COMMON)
 COMMON         0x03000f70     0x13a4 m4aLib.o
                                  0x0 (size before relaxing)
                0x03000f70                m4a_sound
                0x03001f20                ImmSng
                0x03001f90                ImmSngMA
                0x03002010                ExtMPlyJmpTbl
                0x030020a0                m4a_cgbchn
                0x030021a0                ImmSngTA
                0x030022e0                PrsImmSng
 *fill*         0x03002314        0xc
 COMMON         0x03002320     0x1af4 E:\pm3sound20041208\pm3sound\SoundMon.o
                                  0x0 (size before relaxing)
                0x03002320                c_bit
                0x03002324                p_rev
                0x03002328                p_bit
                0x0300232c                c_mvg
                0x03002330                AvrLinC
                0x03002334                c_mvo
                0x03002338                w_midibuf
                0x0300233c                vcount
                0x03002340                Cont
                0x03002344                xcmdn
                0x03002348                MaxLin
                0x0300234c                c_mch
                0x03002350                AvrLinT
                0x03002354                r_midibuf
                0x03002358                Trg
                0x0300235c                c_rev
                0x03002360                sysex
                0x03002364                MaxChnC
                0x03002370                c_song
                0x03002380                c_fre
                0x03002384                p_mch
                0x03002390                midibuf
                0x03002490                IntrMainBuf
                0x03002c90                MaxChn
                0x03002c94                c_mpr
                0x03002ca0                midi_ma
                0x03002ce0                midi_ta
                0x030031e0                runst
                0x030031e4                KeyRep
                0x030031f0                OamBak
                0x030035f0                p_song
                0x03003600                p_fre
                0x03003610                BgBak
                0x03003e10                CurtCurs
 *fill*         0x03003e14        0xc
 COMMON         0x03003e20      0x110 SoundDat.o
                                  0x0 (size before relaxing)
                0x03003e20                m4a_mplay000
                0x03003e60                m4a_mplay001
                0x03003ea0                m4a_mplay002
                0x03003ee0                m4a_memacc_area
                0x03003ef0                m4a_mplay003
                0x03003f30                .=ALIGN(0x4)
                0x03003f30                .=ALIGN(0x4)
                0x03003f30                _end=.
                0x03003f30                _bss_end__=.
                0x03003f30                __bss_end__=.
                0x03003f30                PROVIDE (end, .)

.stab
 *(.stab)

.stabstr
 *(.stabstr)

.stab.excl
 *(.stab.excl)

.stab.exclstr
 *(.stab.exclstr)

.stab.index
 *(.stab.index)

.stab.indexstr
 *(.stab.indexstr)

.comment
 *(.comment)

.debug
 *(.debug)

.line
 *(.line)

.debug_srcinfo
 *(.debug_srcinfo)

.debug_sfnames
 *(.debug_sfnames)

.debug_aranges  0x00000000       0x20
 *(.debug_aranges)
 .debug_aranges
                0x00000000       0x20 C:\Program Files\Cygnus\thumbelf-000512\H-i686-cygwin32\bin/../lib/gcc-lib/thumb-elf/2.9-arm-000512/../../../../thumb-elf/lib/libg.a(memcpy.o)

.debug_pubnames
                0x00000000       0x1d
 *(.debug_pubnames)
 .debug_pubnames
                0x00000000       0x1d C:\Program Files\Cygnus\thumbelf-000512\H-i686-cygwin32\bin/../lib/gcc-lib/thumb-elf/2.9-arm-000512/../../../../thumb-elf/lib/libg.a(memcpy.o)

.debug_info     0x00000000      0x24b
 *(.debug_info)
 .debug_info    0x00000000      0x24b C:\Program Files\Cygnus\thumbelf-000512\H-i686-cygwin32\bin/../lib/gcc-lib/thumb-elf/2.9-arm-000512/../../../../thumb-elf/lib/libg.a(memcpy.o)

.debug_abbrev   0x00000000       0x8b
 *(.debug_abbrev)
 .debug_abbrev  0x00000000       0x8b C:\Program Files\Cygnus\thumbelf-000512\H-i686-cygwin32\bin/../lib/gcc-lib/thumb-elf/2.9-arm-000512/../../../../thumb-elf/lib/libg.a(memcpy.o)

.debug_line     0x00000000      0x1e5
 *(.debug_line)
 .debug_line    0x00000000      0x1e5 C:\Program Files\Cygnus\thumbelf-000512\H-i686-cygwin32\bin/../lib/gcc-lib/thumb-elf/2.9-arm-000512/../../../../thumb-elf/lib/libg.a(memcpy.o)

.debug_frame
 *(.debug_frame)

.debug_str
 *(.debug_str)

.debug_loc
 *(.debug_loc)

.debug_macinfo
 *(.debug_macinfo)

.debug_weaknames
 *(.debug_weaknames)

.debug_funcnames
 *(.debug_funcnames)

.debug_typenames
 *(.debug_typenames)

.debug_varnames
 *(.debug_varnames)

.stack          0x00080000        0x0
                0x00080000                _stack=.
 *(.stack)
OUTPUT(E:\pm3sound20041208\pm3sound\SoundMon.elf elf32-littlearm)
